:020000040800F2
:10000000F85600202902000825340008392B000882
:10001000C5320008D10B0008A94300080000000009
:100020000000000000000000000000001137000880
:100030004914000800000000A1360008393E0008FD
:10004000430200084302000843020008430200087C
:10005000430200084302000843020008430200086C
:10006000430200084302000843020008430200085C
:100070006D13000843020008430200084302000811
:10008000430200084302000843020008430200083C
:10009000D50B0008E50B00084302000843020008E6
:1000A000430200084302000843020008430200081C
:1000B000430200084302000843020008430200080C
:1000C00043020008430200084302000843020008FC
:1000D00043020008430200084302000843020008EC
:1000E00043020008430200084302000843020008DC
:1000F00043020008430200084302000843020008CC
:1001000043020008430200084302000843020008BB
:1001100043020008430200084302000843020008AB
:10012000430200084302000843020008430200089B
:10013000430200084302000843020008430200088B
:10014000F50B0008050C00084302000843020008F4
:10015000430200087D130008430200084302000820
:10016000430200084302000843020008430200085B
:100170004302000843020008430200080000000098
:10018000430200084302000800F002F800F03CF8C7
:100190000AA090E8000C82448344AAF10107DA45E2
:1001A00001D100F031F8AFF2090EBAE80F0013F0F8
:1001B000010F18BFFB1A43F001031847D87E000057
:1001C000F87E0000103A24BF78C878C1FAD85207E8
:1001D00024BF30C830C144BF04680C6070470000C1
:1001E0000023002400250026103A28BF78C1FBD840
:1001F000520728BF30C148BF0B6070471FB507F0DA
:10020000C0FE1FBD10B510BD00F062F91146FFF72A
:10021000F5FF04F073F900F080F903B4FFF7F2FF83
:1002200003BC00F083F900000948804709480047F3
:10023000FEE7FEE7FEE7FEE7FEE7FEE7FEE7FEE796
:10024000FEE7FEE704480549054A064B70470000F3
:10025000F13E000889010008F8500020F8560020FF
:10026000F8520020F852002053EA020C00F0698096
:100270002DE9F04B4FF00006002B1FBFB3FA83F5BA
:1002800003FA05F424FA05F65E4012BF1643B2FAEB
:1002900082F502FA05F4C5F120051EBF22FA05FC1D
:1002A00044EA0C04203556EA044C4FEA144418BFC3
:1002B000641C4FF000084FF00009904271EB030CF2
:1002C00039D3002919BFB1FA81F701FA07F6B0FA5C
:1002D00080F700FA07F6C7F120071EBF20FA07FCD7
:1002E00046EA0C062037B6FBF4FCA7EB0507103FE7
:1002F00007F01F0BCBF120062CFA06F60CFA0BFBCD
:1003000044BFB3460026202FA4BF5E464FF0000B2B
:100310005BEA060C08BF4FF0010B19EB0B0948EB29
:100320000608ABFB027C06FB02CC0BFB03CCC01B1C
:1003300071EB0C01C1E70B46024641464846BDE859
:10034000F08B13B5084318BF4FF0FF300146AFF3F1
:100350000080BDE81C407047032A40F2308010F056
:10036000030C00F0158011F8013BBCF1020F624450
:1003700098BF11F801CB00F8013B38BF11F8013BE1
:10038000A2F1040298BF00F801CB38BF00F8013B8E
:1003900011F0030300F02580083AC0F0088051F8FE
:1003A000043B083A51F804CBA0E80810F5E7121D09
:1003B0005CBF51F8043B40F8043BAFF30080D20728
:1003C00024BF11F8013B11F801CB48BF11F8012BF4
:1003D00024BF00F8013B00F801CB48BF00F8012B17
:1003E000704710B5203AC0F00B80B1E81850A0E873
:1003F0001850B1E81850A0E81850203ABFF4F5AFF3
:100400005FEA027C24BFB1E81850A0E8185044BF4E
:1004100018C918C0BDE810405FEA827C24BF51F8BB
:10042000043B40F8043B08BF7047D20728BF31F8AF
:10043000023B48BF11F8012B28BF20F8023B48BF00
:1004400000F8012B704702F0FF0343EA032242EA5F
:10045000024200F002B84FF0000200B51346944685
:100460009646203922BFA0E80C50A0E80C50B1F10C
:100470002001BFF4F7AF090728BFA0E80C5048BF20
:100480000CC05DF804EB890028BF40F8042B08BFBE
:10049000704748BF20F8022B11F0804F18BF00F8BA
:1004A000012B704770477047704710B500F008F88F
:1004B000006810BD10B5044600F002F8046010BDDD
:1004C00000487047C800002000487047C80000205E
:1004D0007546FFF7F9FFAE4605006946534620F022
:1004E0000700854618B020B5FFF7ACFEBDE82040F8
:1004F0004FF000064FF000074FF000084FF0000BE0
:10050000AC46ACE8C009ACE8C009ACE8C009ACE84E
:10051000C00921F007018D46704710B50446AFF3BE
:1005200000802046BDE81040FFF777BE0149182043
:10053000ABBEFEE72600020070470000B1EE601A75
:10054000B4EE600AF1EE10FAB4EE401AC8BFB0EE95
:10055000600AF1EE10FAC8BFB0EE410A7047000021
:100560002DE9F04381B040F64C18C2F2000806466F
:10057000D8F8000014460D466421002A08BF0A245A
:1005800004F04EF908B1FB242FE040F64819C2F2FE
:100590000009D9F8000000E0006930B10178B142EB
:1005A000FAD14168A942F7D11AE0142000F0BAFA52
:1005B00088B1074620461C21002204F099F8B86053
:1005C00058B1D9F800003C7300243E707D6038615A
:1005D000C9F8007005E0FE2403E0384600F09EFAFA
:1005E000FF24D8F8000004F091F960B201B0BDE832
:1005F000F08300007047000040F64812C2F200028B
:10060000126800E01269002A04BF002070471378C6
:100610008342F7D153688B42F4D190687047000051
:10062000D0E90212081FB0FA80F14FF0020008BFB3
:100630000320022A18BF48097047000040F25C22DC
:1006400040F23421C2F200020128C2F2000118BFB8
:100650000022002818BF1146012888BF0021084643
:10066000704700002DE9F041154640F2D832C2F241
:1006700000021278012A11D1A5B140F64C18C2F23D
:1006800000080746D8F800000E4664211C4604F016
:10069000C7F858B1FB2040B2BDE8F081FD2040B260
:1006A000BDE8F081FE2040B2BDE8F0813846314619
:1006B000FFF7A2FFD8F800100646084604F026F916
:1006C00066B1304629460022234603F0CDFF0028BC
:1006D00018BF4FF0FF3040B2BDE8F081FC2040B2BF
:1006E000BDE8F0812DE9F0438BB040F2D836C2F27C
:1006F0000006307808B1FD275EE040F22810C2F213
:1007000000006821FFF7A7FE40F2D43040F2F55117
:10071000C2F20000C0F6000101600020002704F0D2
:10072000A9F840F64C11C2F200010028086042D03E
:100730000DF104080124404628213470FFF78BFE98
:1007400040F23425C2F200054FF00E09284641461A
:10075000CDE90377CDE90844CDF82890059700F05E
:10076000D7FE284601F092FA40F63902C0F60002A0
:100770000020062100F02EF82846032100F06AFE32
:1007800040F25C25C2F2000528464146CDE9054904
:1007900000F0BEFE284601F079FA40F6FD02C0F6F0
:1007A00000020120082100F015F82846102100F071
:1007B00051FE347000E0FF2778B20BB0BDE8F08343
:1007C00080B540F2D432C2F200021268002A18BF8B
:1007D000904780BD40F2D833C2F200031B78012B52
:1007E0001EBFFD2358B270473AB101284FF0FF03F6
:1007F00098BF0C2904D958B27047FE2358B27047ED
:1008000040F2281CC2F2000C342310FB03C000236A
:1008100040F8212058B2704780B540F2D833C2F278
:1008200000031B78012B03D1FFF79AFE40B280BD75
:10083000FD2040B280BD00002DE9F04F93B003A829
:100840000D3001904FF0000A0CAE002005E000BF13
:100850000298002800F101004CD15FFA80FB029061
:100860005846FFF7EBFE0028F2D0044609E000BF2F
:1008700001F0E6FC0990384603A90022002303F0AA
:1008800087FF2046002100F0C5FE0028E0D020466A
:10089000002132460AAB00F0CDFE0028F1D10E98BF
:1008A0000028304618BF043005683046FFF7B8FE10
:1008B000804628464146FFF783FF81465846494611
:1008C000FFF79AFE0028DCD00746DDE90F02CDF8DD
:1008D0000CA00028CDE908AACDE906AA8DF80C8065
:1008E000CDE904598DF81820C2D101980AA9FFF763
:1008F00033FDBDE713B0BDE8F08F00002DE9F04FE8
:1009000093B003A80D3001904FF0000A0CAE002008
:1009100005E000BF0298002800F101004CD15FFA09
:1009200080FB02905846FFF789FE0028F2D004466B
:1009300009E000BF01F084FC0990384603A90022B9
:10094000002303F025FF2046012100F063FE00286C
:10095000E0D02046012132460AAB00F06BFE0028B1
:10096000F1D10E980028304618BF04300568304693
:10097000FFF756FE804628464146FFF721FF814695
:1009800058464946FFF738FE0028DCD00746DDE927
:100990000F02CDF80CA00028CDE908AACDE906AADF
:1009A0008DF80C80CDE904598DF81820C2D101983A
:1009B0000AA9FFF7D1FCBDE713B0BDE8F08F000036
:1009C000F0B587B0154640F2D832C2F20002127874
:1009D000012A03D1012803D9FF203EE0FD203CE09D
:1009E0000E4601F0FE011C46022902D00CB9FE2081
:1009F00033E00C9F082F01D9FF202EE0FFF71EFEE9
:100A000080B10021032E0691CDE90411CDE9021138
:100A1000019125D8DFE806F002080B0F01950022AE
:100A200000210BE0FE2018E00295002105E0019571
:100A30000221002202E0022102950422CDE90321D5
:100A400000218DF8181001A96B462246059700F089
:100A500015FD002818BF4FF0FF3040B207B0F0BDC1
:100A6000FF20FAE779B180B582B00A6891F804C036
:100A70004B1D0021CDF800C0FFF7A2FF02B0BDE87A
:100A8000804040B27047FE2040B270472DE9F043ED
:100A900081B040F2D832C2F200021278012A03D1AA
:100AA000012806D9FF2700E0FD2778B201B0BDE894
:100AB000F0830C46FFF7C2FD20B3054601F0C0FBF2
:100AC00014B3804604F1010904E000BF00260027AA
:100AD000002EEAD0284600F03FFE0028F6D1B9F1FA
:100AE000000F08D001F0ACFBA0EB0800A04228BF2B
:100AF0006FF0040704D20120012603F017FDE7E799
:100B00000026E5E7FE27D0E7284600F025FE00276F
:100B1000002808BF6FF00407C7E7000080B504F0A5
:100B200073FE80BD80B504F0F9FC80BD2DE9F04175
:100B300003F030FD044606F021F84FF47A784EF2C7
:100B40001806B8FBF4F4CEF20006376804FB00F593
:100B500006F014F860433168854208BF394656F8FC
:100B6000042C01FB08F10132B1FBF2F100FB08F0AB
:100B7000401A00F57A700021BDE8F08140F28C3215
:100B800040F24431C2F200020128C2F2000118BF53
:100B90000022002818BF1146084670473AB10128C4
:100BA0004FF0FF0398BF082904D958B27047FE23BD
:100BB00058B2704740F2981300EBC000C2F2000335
:100BC00003EB8000002340F8212058B2704700005A
:100BD000FEE7000080B540F23420C2F2000000F0D1
:100BE000CFFD80BD80B540F23420C2F2000000F09D
:100BF000C7FD80BD80B540F25C20C2F2000000F06D
:100C0000BFFD80BD80B540F25C20C2F2000000F064
:100C1000B7FD80BD4FF0030160B146F200420068AD
:100C2000C4F2000202F58063984208BF0121801AD5
:100C300008BF0146C8B2704700284FF0FF0218BF36
:100C4000002901D150B2704780B590ED010A9FEDA7
:100C5000793A90ED021A30EE030A9FED773A9FED54
:100C6000775A30EE000A90ED032A80EE036A31EEE7
:100C7000050A9FED731A9FED735A30EE000A90ED4E
:100C8000044A80EE011A32EE050A9FED6F2A9FEDAD
:100C90006F5A30EE000A80EE022A34EE050A30EE7A
:100CA000000A80EE035ABFEE000A36EE006A81EDBC
:100CB000016A31EE004A81ED024AB0EEC44A32EEDA
:100CC000003A9FED632A81ED033A35EE001AB0EE4B
:100CD000C65AB4EE425AF1EE10FAB4EE424AB0EE01
:100CE000C33A81ED041ADCBF00224A60F1EE10FA2B
:100CF000B4EE423AB0EEC11ADCBF00228A60F1EED7
:100D000010FAB4EE421ADCBF0022CA60F1EE10FA0B
:100D1000DCBF00220A6191ED012AB7EE001AB0EEA5
:100D2000C23AB4EE413AF1EE10FA0ADBB5EE402ACF
:100D3000B0EE402AF1EE10FAC8BFB0EE412A81EDC4
:100D4000012A91ED022AB0EEC23AB4EE413AF1EE38
:100D500010FA0ADBB5EE402AB0EE402AF1EE10FAA6
:100D6000C8BFB0EE412A81ED022A91ED032AB0EE10
:100D7000C23AB4EE413AF1EE10FA0ADBB5EE402A7F
:100D8000B0EE402AF1EE10FAC8BFB0EE412A81ED74
:100D9000032A91ED042AB0EEC23AB4EE413AF1EEE4
:100DA00010FA08DBB5EE402AF1EE10FAC8BFB0EE3B
:100DB000410A81ED040AD1E9032301F11407D1E9C5
:100DC00001CE87E80C5090F800E0BEF1000F02D091
:100DD000C37E012B20D100234B70807D831EB3FA8C
:100DE00083F35A09431EDBB2022B8A700AD8DA0059
:100DF0004FF0011323FA02F2012881F8242001D1D7
:100E0000012000E00020002281F8250081F800E0A8
:100E1000BDE8804050B27047037E013BDBB2022B3D
:100E2000DBD84FEAC30C40F20313C0F2020323FAEB
:100E30000CF3D1E7000051C30060AD44000032C3A1
:100E40000020AC44000052C30040AD4400005DC32C
:100E5000CDCC4C3D00000000002800F08D802DE935
:100E6000F0412DED088B9FED66AA9FED66BA804696
:100E700000250A264FF416772024B7EE009ABFEE1D
:100E8000008A25E008EB040090ED000A08EB07005B
:100E900001F054FE80EE0B1A08EB050080ED130AFA
:100EA0000435083620371034B4EE491AF1EE10FA42
:100EB000C8BFB0EE491AB4EE481AF1EE10FAB8BF46
:100EC000B0EE481A3AEE01AA042D80ED171A18D197
:100ED000D8F81400304402F095F8D8F814003044E3
:100EE00001F0AAFF0028CDD000F12C0C08EB850101
:100EF0009CE80C10806B01F11C0E8EE80C108862CF
:100F0000C0E7D8F81400B6EE000A2AEE000A1A303C
:100F100088ED190A02F076F8D8F814001A3001F0BA
:100F20008BFF48B100F108030ECB406908F13C0C7F
:100F30008CE80E00C8F8480098ED0F0A10EE100A71
:100F400088ED160A06F07CFF41EC100B9FED2A1B82
:100F500006F0FEF851EC100B06F008FB9FED2B1A83
:100F600000EE100AB4EE410AF1EE10FAC8F858008B
:100F700005DD9FED251A0BE0FF2040B270479FED85
:100F8000251AB4EE410AF1EE10FA05DA9FED201AA7
:100F900031EE000A88ED160A98ED100A08F5367051
:100FA00001F0CCFD98ED101A9FED1B2A88ED150A73
:100FB00081EE021A98ED080A98ED0C2A002030EE16
:100FC000420AB4EE491AF1EE10FAC8BFB0EE491A5F
:100FD000B4EE481AF1EE10FAB8BFB0EE481A88ED38
:100FE0001A1A88EDC60ABDEC088BBDE8F04140B284
:100FF000704700BF00BF00BF00000060FB21194028
:101000000000000000C0DA45DB0FC9C0DB0F49401B
:10101000DB0FC940DB0F49C000409C45B5EE401ACC
:10102000F1EE10FA30EE600AD8BF7047B6EE002A33
:1010300021EE022AB4EE420AF1EE10FAC4BF30EEFD
:10104000410A7047B1EE422AB4EE420AF1EE10FABC
:10105000B8BF30EE010A704740F20400C2F200004F
:1010600070470000B0B5E8B140F2D934C2F20004D4
:10107000207810B1FD2568B2B0BD03F005FD40F643
:101080001051C2F20001086060B141F22532C0F691
:101090000002002003210025FFF780FD01202070C1
:1010A00068B2B0BDFE2568B2B0BD00002DE9F04FBA
:1010B00082B090F802C0C27840F650134FEADC04C8
:1010C000C2F2000362F34A1490F8019005795C8043
:1010D000C2784679AD0045EA921206F0010542EA6F
:1010E00085229A80457987796E0867F3CA16DE8073
:1010F0008579C7794FEA151E67F30A1EA3F808E041
:10110000077A90F80780457A7F0047EAD81705F0FC
:10111000030547EA452BA3F80AB0457A877A4FEAD8
:10112000950867F38A18A3F80C80C77A857AFF00C0
:1011300047EA5515DD8190F80CA0477B009567F3D1
:101140000A2AA3F810A0477B857BFF0865F34A179E
:101150005F820197C77B6CF30A2990F80EC0057C6B
:10116000BF0047EA9C1705F0010547EA852CA3F864
:1011700014C0057C477C680800EE104A01EE102A76
:1011800002EE106AAEF22D1203EE109A67F3CA1047
:10119000C72AB8EEC33AB8EEC00AB8EEC11AB8EE24
:1011A000C22AA3F80090D88281ED012A81ED021AAB
:1011B00081ED033A81ED040A01D201220DE0AEF582
:1011C000FA72B2F57A7F01D2032206E0AEF2DC5267
:1011D0000023C82A38BF01235A00ABF22D13DDE9E2
:1011E00000679BB2C72B0A7501D201220FE0ABF555
:1011F000FA7292B2B2F57A7F01D2032207E0ABF223
:10120000DC5292B20023C82A38BF01235A00A8F248
:101210002D13C72B4A7501D201220DE0A8F5FA72F1
:10122000B2F57A7F01D2032206E0A8F2DC52002355
:10123000C82A38BF01235A00A6F22D13C72B8A757E
:1012400001D202220CE0A6F5FA72B2F57A7F01D241
:10125000032205E0A6F2DC530022C82B38BF01228E
:10126000AAF22D13C72BCA7501D202220CE0AAF5EF
:10127000FA72B2F57A7F01D2032205E0AAF2DC53BA
:101280000022C82B38BF0122A7F22D13C72B0A76E4
:1012900001D202220CE0A7F5FA72B2F57A7F01D2F0
:1012A000032205E0A7F2DC530022C82B38BF01223D
:1012B000ACF22D139BB2C72B4A7601D201220FE06C
:1012C000ACF5FA7292B2B2F57A7F01D2032207E04E
:1012D000ACF2DC5292B20023C82A38BF01235A0074
:1012E000A0F22D13C72B8A7601D202220CE0A0F5C2
:1012F000FA72B2F57A7F01D2032205E0A0F2DC5344
:101300000022C82B38BF0122B0F59670CA7618BFEC
:101310000120B9F57A7218BF01221040087002B09E
:10132000BDE8F08F80B540F61050C2F200000068B2
:10133000802103F00BFB80BD10B504460020FFF7B1
:101340001DFC2146192201F0B9FB002818BF4FF0FF
:10135000FF3010BD80B502468020012103F036FB2E
:101360008038B0FA80F0400980BD000080B540F2BE
:101370008420C2F2000000F035FD80BD80B540F24F
:10138000E420C2F2000000F02DFD80BDD0F800C0C6
:101390006FF00F024AF6AB2352FA8CF2CAF6AA2378
:1013A0000146A2FB0330000905A31B5C40F2FF309D
:1013B0002CEA00005F2A88BF0430C1E91603704799
:1013C00000061016000610168269816AB2F5005FE9
:1013D00006D06AB9022912D0012914D0D1B90EE081
:1013E000032917D8DFE801F0020B020F0120704734
:1013F00003293CBF012070471CBF00207047C06A12
:10140000C0F300607047C06AA0F1C070B0FA80F00D
:10141000400970470020704780B5D0F800C0D0F870
:1014200008E0DCF80000BEF1400F20F48020CCF88A
:1014300000000846CCF8043004BF10460A46CCF839
:101440000800CCF80C2080BD7047000072B600BFC9
:10145000FEE7000090F82020013A012A04D8006835
:1014600000F11402002004E000F1240201204FF4F6
:1014700080211368194311607047000010B590F87F
:1014800020E0D0F800C0AEF1010EBEF1010FDCF893
:1014900008E00ED81EF0E05F11D0CEF3016E0120FF
:1014A00000FA0EF018608B687BB1486843EAC0030D
:1014B0000DE000F1240101204FF4802223E000F12F
:1014C000240101204FF400121DE008684305D1E912
:1014D000030403430CEB0E10C0F88031C0F88441C4
:1014E000097D012905D100F5C2710B6843F48073B1
:1014F0000B605168C0F88C11126800F5C071C0F81B
:101500008821002001220B681A430A6010BD0000E8
:10151000B0B590F82020013A012A2FD846F2006099
:10152000C4F20000026842F001020260026822F484
:101530007C520260D1F814E0CC694A6A0368012C3D
:1015400043EA022202600EF01F024FF0010303FA89
:1015500002F2C3696FEA020C23EA0203C36113D0EB
:101560002CBBC36803EA0C03C360CB688C8844EAD5
:10157000034300EBCE0423640B4611E0416A41F4BF
:10158000802141620120B0BDC3681343C3600B6872
:101590008C8844EA034300EBCE04236401F10C037E
:1015A0008C681B8843EA044300EBCE046364436801
:1015B0008D6943EA0204D1F810E0096A002D08BFE2
:1015C00003EA0C0444604369BEF1000F43EA0204DD
:1015D00008BF03EA0C040129446102D1C169114327
:1015E000C161016821F0010101600020B0BD00006F
:1015F00080B5FFF70FFB032808BF80BD40F228111C
:10160000C2F20001342210FB0210006B002818BF48
:10161000804780BD90F82020013A012A84BF002035
:10162000704700681022002908BF0C22805800F083
:101630000300704710B590F82040013C012C0AD8F7
:10164000046871B12469A4070ED100F124010120BE
:101650004FF4001276E000F1240101204FF48022C3
:1016600070E0E468A40771D0046804EB011CDCF8A6
:10167000B0410CF5D87E14F004049460DCF8B0415D
:1016800019BFE4085460640D1460DEF800400CF5E6
:10169000DA7E04F00204D460DCF8B44124075ABFB7
:1016A000DEF8004004F00F0408241461DEF8004066
:1016B0000029C4F307249461DEF800404FEA144483
:1016C0005461DCF8B8211A70026802EB0112D2F8FA
:1016D000B8214FEA12225A70026802EB0112D2F8C6
:1016E000B8214FEA12429A70026802EB0112D2F856
:1016F000B8214FEA1262DA70026802EB0112D2F8E6
:10170000BC211A71026802EB0112D2F8BC214FEA27
:1017100012225A71026802EB0112D2F8BC214FEA80
:1017200012429A71026802EB0112D2F8BC214FEA10
:101730001262DA71006814BF00F1100100F10C01AF
:10174000002020220B681A430A6010BD00F124011A
:1017500001204FF40012F5E790F82010013901291B
:1017600084BF002070470068816882688068C1F388
:101770008061C2F3C0621144C0F300700844704736
:101780002DE9F04F81B0044600684669D0F8049016
:101790008768D0F80CB0D0F810A0D0F81880F10706
:1017A00003D1002530071CD423E0F90710D0012114
:1017B000BA07816009D4780700F1AA80380700F1E0
:1017C000B080204600F090FA02E0204600F09EFA39
:1017D0000025F80500F18480F80300F1AA803007A5
:1017E00007D51BF0100004D0206845F400751021C7
:1017F000C160700708D51BF0080005D020680821DB
:10180000C160204600F0E8F9B00706D52068C0683E
:10181000800702D0204600F0F1F9700607D51AF0D3
:10182000100004D0206845F4806510210161B006E5
:1018300008D51AF0080005D020680821016120466B
:1018400000F0EEF9F00606D520680069800702D0A6
:10185000204600F0F7F9B00308D519F0100005D0C4
:10186000206810214160204600F0FEF9F00308D501
:1018700019F0080005D0206808214160204600F0DA
:101880009FFA300440F18F805FEA497040F1888010
:1018900006F4807008EA102028435FEA8871014648
:1018A00048BF41F00201B20558BF01465FEA4870E7
:1018B0000D4648BF45F00405700558BF0D4630057C
:1018C0006ED518F070006BD010380009052862D86A
:1018D000DFE800F0035356595C5F45F008055AE015
:1018E00020684FF48071BA0581600AD4780512D45B
:1018F000380519D4204600F01BFAF8037FF56FAFC6
:1019000017E0204600F026FAF8037FF568AF10E0F4
:101910004FF400655DE705F50055F8037FF55FAF0F
:1019200007E04FF4805554E705F58045F8037FF54F
:1019300056AF20684FF48031BA0381600AD478032F
:101940000FD4380313D4204600F016FA30073FF5C1
:1019500048AF4EE7204600F021FA30073FF541AF8F
:1019600047E705F5004530073FF53BAF41E705F593
:10197000803530073FF535AF3BE745F010050AE00D
:1019800045F0200507E045F0400504E045F08005FE
:1019900001E045F480752068816921F07001816162
:1019A0002068042141602DB1606A284360622046AE
:1019B000FFF71EFE01B0BDE8F08F0000B0B5C8B162
:1019C000044690F8200010B9204600F071F8206815
:1019D000016841F00101016000F032FC054600BFE2
:1019E00020684168C90707D100F02AFC401B0B287A
:1019F000F6D312E00120B0BD016821F002010160C0
:101A000000F01EFC054600BF2068416889070DD51F
:101A100000F016FC401B0B28F6D3606A052140F449
:101A200000306062012084F82010B0BD217E026881
:101A3000012922F0800208BF80320260617E0268C4
:101A4000012922F0400208BF40320260A17E0268F4
:101A5000012922F0200208BF20320260E17E0268E4
:101A6000012922F0100218BF10320260217F0268A3
:101A7000012922F0080208BF08320260617F026873
:101A8000012922F0040208BF04320260D4E901C235
:101A9000D4E9033561691A432A431143ACF10102C9
:101AA0001143C16100200121606284F82010B0BDA3
:101AB000B0B586B0006846F60002C4F2000200210C
:101AC0009042CDE90411CDE9021101912FD046F2E7
:101AD0000041C4F2000188427BD140F29011C2F271
:101AE00000010A6843F64000C4F20200531C0B6078
:101AF00052B900210091016841F000710160016854
:101B000001F00071009100990021009150F8101C23
:101B1000152441F0020140F8101C50F8100C142557
:101B200000F00200009000984FF4407031E043F65E
:101B30004000C4F202000091016841F08061016040
:101B4000016801F080610091009940F29011C2F2A9
:101B500000010A68531C0B6052B900210091016812
:101B600041F000710160016801F00071009100997D
:101B70000021009150F8101C412441F0020140F86E
:101B8000101C50F8100C402500F002000090009846
:101B90006020019002200290002003900320049016
:101BA0000920059040F20040C4F2020001A900F0B3
:101BB00079FA28460521002200F0C2FB284600F0F1
:101BC000BBFB20460521002200F0BAFB204600F0B6
:101BD000B3FB06B0B0BD000080B5FFF71BF80328CB
:101BE00008BF80BD40F22811C2F20001342210FB70
:101BF0000210C069002818BF804780BD80B5FFF77C
:101C000009F8032808BF80BD40F22811C2F2000184
:101C1000342210FB02108069002818BF804780BD65
:101C200080B5FEF7F7FF032808BF80BD40F22811FA
:101C3000C2F20001342210FB0210406A002818BFD3
:101C4000804780BD80B5FEF7E5FF032808BF80BD53
:101C500040F22811C2F20001342210FB0210006A87
:101C6000002818BF804780BD80B5FEF7D3FF03284A
:101C700008BF80BD40F22811C2F20001342210FBDF
:101C80000210806A002818BF804780BDB0B50446A6
:101C900090F8200001281DD1022084F8200020683F
:101CA000016821F00101016000F0CAFA054600BF99
:101CB00020684068C00713D000F0C2FA401B0B2810
:101CC000F6D3606A40F400306062052084F820009A
:101CD0000120B0BD606A40F4002060620120B0BD08
:101CE00000206062B0BD000080B5FEF793FF0328BE
:101CF00008BF80BD40F22811C2F20001342210FB5F
:101D00000210C068002818BF804780BD80B5FEF76C
:101D100081FF032808BF80BD3421484340F22811C9
:101D2000C2F200010858002818BF804780BD00009B
:101D300080B5FEF76FFF032808BF80BD40F2281171
:101D4000C2F20001342210FB02100069002818BF03
:101D5000804780BD80B5FEF75DFF032808BF80BDCA
:101D600040F22811C2F20001342210FB0210406838
:101D7000002818BF804780BD80B5FEF74BFF0328C1
:101D800008BF80BD40F22811C2F20001342210FBCE
:101D900002104069002818BF804780BD80B5FEF75B
:101DA00039FF032808BF80BD40F22811C2F20001AC
:101DB000342210FB02108068002818BF804780BDC5
:101DC00080B5FEF727FF032808BF80BD40F2281129
:101DD000C2F20001342210FB0210C06A002818BFB2
:101DE000804780BDF0B581B004460020009040F2ED
:101DF0000000C2F200000268D4E9166048F2B51390
:101E000037680821C1F64E3381403942A2FB0325D1
:101E10000CD0226813685B0708D5136823F004030D
:101E20001360B160616D41F0010161650121814084
:101E3000394208D022685269120604D5B160616D3A
:101E400041F00201616504218140394208D02268D5
:101E50001268920704D5B160616D41F004016165BB
:101E600010218140394215D020680268120711D52F
:101E7000B16002680168520306D4C90506D401683E
:101E800021F00801016001E0080342D4216C09B18E
:101E900020468847E16D202000FA01F23A4244D002
:101EA00020680368DB0640D5B26094F835300268DC
:101EB000052B1ED122F016020260426922F0800238
:101EC0004261226C0AB9A26C1AB1026822F00802BF
:101ED00002603F208840B060012084F83500216D09
:101EE0000020002984F8340040D02046884701B003
:101EF000F0BD0168520310D4C90512D4016821F065
:101F000010010160012084F83500002084F83400BD
:101F100007E0A16C0029BBD1BCE7080301D4616CC8
:101F200000E0E16B09B120468847606DF0B1606D5B
:101F3000C00717D0052084F835002068A90A026878
:101F400022F00102026000BF009A01328A42009230
:101F500002D80268D207F7D1012084F835000020AA
:101F600084F83400E16C09B12046884701B0F0BD27
:101F70002DE9F041044600F063F9C4B105460220A2
:101F800084F835000020216884F83400086820F0C7
:101F90000100086026683068C0070BD000F050F9D7
:101FA000401B0528F6D903212022032042E001200E
:101FB000BDE8F081306848F23F01CFF21001251DE5
:101FC00000EA010C2ECDD4E9050E41EA0C011143C3
:101FD00019432943D4E90778084340EA0E01606AAF
:101FE0003943042841EA080103D1D4E90B23114302
:101FF000194331607169042821F0070141EA0005A5
:102000000CD1D4E90A1045EA010538B12046FFF7A2
:10201000DBF918B10121402201200BE02046756157
:10202000FFF7B4F9E16D3F2202FA01F1816000226D
:1020300001210020626584F83510BDE8F0810000C0
:10204000B0B5044690F83400012828D0012084F867
:102050003400A56D94F8350001281DD1022084F8C4
:102060003500002060652046FFF7D6F9E26D3F237A
:10207000206803FA02F2216CAA60026842F016029C
:10208000026019B1016841F008010160016841F086
:10209000010101600020B0BD002084F8340002205E
:1020A000B0BD00002DE9F04F83B000F13E4202F1D7
:1020B000FF724FEAB22241F600470192C4F20207D2
:1020C00008224FF0010E00254FF0000A4FF00008E3
:1020D000B84208BF072200920AE000BF08F10108D9
:1020E0000AF1040AB8F1100F05F1020500F0A4800E
:1020F0000C680EFA08FB14EA0B09EFD04C6804F0E8
:10210000030CACF1010EBEF1010F11D80322876858
:1021100002FA05F6CA68B743AA403A4382604268A9
:10212000C4F3001722EA0B0207FA08F73A434260A9
:10213000BCF1030F1CD0C26803238E6803FA05F7B5
:10214000BA4306FA05F73A43BCF1020FC2600FD159
:102150006FF0030202EA580202440AF01C060F2341
:10216000176A03FA06F40B69A743B3403B431362B3
:10217000026803234F68AB409A4307F00303AB4068
:102180001A4317F4403F4FF0010E0260A6D0002220
:1021900043F644030292C4F202031A6843F6004471
:1021A00042F480421A601A68C4F2010402F48042C8
:1021B0000292029A28F003024FF6084B2244CFF60F
:1021C000FF7B52F80B300AF00C070F26BE4023EAC3
:1021D000060C019B009E072B38BF1E4606FA07F728
:1021E00047EA0C0342F80B30A2684B6842EA090741
:1021F00043F60C4CDE0258BF22EA0907A760C4F27E
:10220000010CDCF800209E0242EA090758BF22EACE
:102210000907CCF8007062689E0342EA090758BFBC
:1022200022EA090767602268DB0342EA090358BF14
:1022300022EA0903236051E703B0BDE8F08F0000F4
:1022400044F61C10C2F200000068704740F2B8006B
:1022500044F61C11C2F20000C2F2000100780A68C4
:10226000104408607047000080B543F60040C4F297
:102270000200016841F400710160016841F480616D
:102280000160016841F480710160032000F068F88A
:102290000F2000F005F800F02BF8002080BD0000B2
:1022A000B0B540F2B802C2F2000240F2000112786A
:1022B000C2F200014FF47A730968B3FBF2F20446EC
:1022C000B1FBF2F1084600F001FB0F2C4FF00105C5
:1022D0000CD858B94FF0FF3021460022002500F0FD
:1022E0002FF840F2BC00C2F2000004602846B0BDE6
:1022F00080B582B0002043F640010190C4F2020193
:102300004A6842F480424A604A6802F4804201927C
:10231000019A00900868002240F080500860086828
:102320000F2100F08050009000986FF0010000F045
:1023300007F802B080BD000080B502F04FF880BD04
:1023400070B514460D46064602F058F82946224656
:1023500001F06AF80146304602F058F870BD0000FE
:1023600080B502F06DF880BD2DE9F041002800F045
:102370008B8043F60808C4F202080446D8F8F80334
:102380000D4600F00700884207D288F8F853D8F8C5
:10239000F80300F00700A84276D12068810717D51E
:1023A000410705D5D8F8001041F4E051C8F80010F5
:1023B000010705D5D8F8001041F46041C8F80010B5
:1023C000D8F80010A26821F0F0011143C8F80010FD
:1023D000C0073FD1D8F8F80300F00700A84207D99A
:1023E00088F8F853D8F8F80300F00700A8424BD15A
:1023F0002068410707D5D8F80010E26821F4E051C1
:102400001143C8F80010000708D5D8F8000021696A
:1024100020F4604040EAC100C8F8000000F07EF8F7
:10242000D8F8001047F6C872C1F30311C0F60002D5
:10243000515C40F2000220FA01F140F2BC00C2F20D
:1024400000000068C2F200021160FFF729FF0020BF
:10245000BDE8F0816068811E022907D258F8081C87
:1024600089015CBF0120BDE8F08110E0012807D19F
:1024700058F8081C89035CBF0120BDE8F08106E024
:1024800058F8081C890702D40120BDE8F081D8F86B
:10249000001021F003010843C8F80000FFF7D0FE48
:1024A000064641F2883700BFD8F80000616800F0A6
:1024B0000C00B0EB810F8DD0FFF7C2FE801BB8423D
:1024C000F2D90320BDE8F08140F20000C2F2000022
:1024D0000068704780B5FFF7F7FF43F60801C4F2C4
:1024E0000201096847F6D872C1F38221C0F60002E2
:1024F000515CC84080BD000080B5FFF7E5FF43F6A2
:102500000801C4F20201096847F6D872C1F34231EA
:10251000C0F60002515CC84080BD000010B543F613
:102520000404C4F20204606800F00C0008280AD019
:10253000042819BF42F20040C0F2F40041F6003016
:10254000C0F2B70010BD206821682368490241F637
:102550000031C0F2B70100F03F02C3F388105CBF46
:1025600042F20041C0F2F401A1FB00010023FDF79B
:102570007BFE21680222C1F3014102EB4101B0FB65
:10258000F1F010BD2DE9F04182B0002800F0A280EA
:102590000446007843F60006C007C4F2020643D0A2
:1025A000B06800F00C00042805D1306880033BD5EA
:1025B0006068C8BB8EE0B06800F00C00082802D14B
:1025C00070684002F1D46568B5F5A02F0AD0B5F562
:1025D000803F0BD0306820F480303060306820F4C9
:1025E000802006E0306840F480203060306840F49D
:1025F00080303060FFF724FE002D054611D000BF6B
:102600003068800310D4FFF71BFE401B6428F7D905
:1026100022E100BFFFF714FE401B64284FF00300C7
:1026200055D830688003F5D4207880071AD5B06873
:1026300010F00C0F09D0B06800F00C00082840F032
:102640008A807068400200F186803068800702D579
:10265000E06801283ED13068216920F0F80040EAA6
:10266000C10030602078000738D4207840074CD46F
:10267000A5695DB3B06800F00C00082840F09E80AA
:10268000012D27D07068E16900F480028A4221D1CF
:10269000216A00F03F028A421CD147F6C071626A8B
:1026A0000140B1EB821F15D1A26A0023CFF6FF7360
:1026B00003EBC23200F440316FF30F02914209D1B3
:1026C000E16A00F07060B0EB016F03D1002002B04E
:1026D000BDE8F081012002B0BDE8F081606900280A
:1026E00040F20000C4F2472057D00121C0F8801EFC
:1026F000FFF7A6FD054600BF706F8007B5D4FFF752
:102700009FFD401B0228F7D9A6E0306C10F08058DE
:102710000AD100200190306C40F080503064306C61
:1027200000F080500190019847F20007C4F20007C2
:102730003868C00524D4386840F480703860FFF7EA
:102740007FFD05463868C0051AD4FFF779FD401BA8
:102750000228F7D980E0E068002851D00020C4F2B8
:10276000472001210160FFF76BFD054630688007B7
:102770003FF571AFFFF764FD401B0228F6D96BE00F
:10278000A568052D50D0012D52D0306F20F00100EA
:102790003067306F20F004004DE00021C0F8801E4B
:1027A000FFF74EFD054600BF706F80077FF55DAFF8
:1027B000FFF746FD401B0228F6D94DE00027C4F282
:1027C000472700203866FFF73BFD022D05460BD159
:1027D0003068800158D5FFF733FD401B02284FF0C9
:1027E0000300F5D973E700BF306880017FF56EAF55
:1027F000FFF726FD401B02284FF00300F4D966E7DF
:102800000020C4F2472000210160FFF719FD0546B2
:10281000306880077FF526AFFFF712FD401B0228C6
:102820004FF00300F4D952E7306F40F004003067F6
:10283000306F40F001003067FFF702FD002D0546C4
:1028400041F2883714D000BF306F800713D4FFF7F0
:10285000F7FC401BB842F7D9032002B0BDE8F08175
:10286000FFF7EEFC401BB8424FF003003FF62FAFDE
:10287000306F8007F4D4B8F1000F7FF4F9AE306CFC
:1028800020F080503064F3E604F11C052FCD08439E
:102890000021CFF6FF7140EA821001EBC3316FF3E4
:1028A0000F0140EA05600843706001203866FFF7B9
:1028B000C7FC0446306880013FF508AFFFF7C0FC55
:1028C000001B02284FF00300F4D900E780B501F0A7
:1028D0009BFA80BD7047000080B501F091FC032891
:1028E00008BF80BD40F2981100EBC000C2F20001A9
:1028F00001EB80000069002818BF804780BD000000
:10290000002804BF0120704710B5044690F841002C
:1029100028B9002084F84000204600F021F8242047
:1029200084F841002068C16821F40051C16020464C
:1029300001F076FC2068016921F490410161416950
:1029400021F02A014161C16841F40051C1600020B9
:102950002021606484F8411084F84210606310BD47
:1029600070B586B00446006841F20041C4F201012E
:1029700000268842CDE90466CDE9026601964ED074
:1029800044F60001C4F20001884240F09580002620
:1029900043F630000096C4F20200016941F4802140
:1029A0000161016901F4802100910099009601689C
:1029B00041F004010160006801A900F004000090EA
:1029C00000984FF4406001900220CDE902060320F8
:1029D00004900720059040F60000C4F20200FFF7C3
:1029E00061FB40F2842546F22800C2F20005C4F2E1
:1029F00002004FF000614FF4806285E843002846F2
:102A0000C5E90362C5E90566C5E907666E62FFF7B9
:102A1000AFFA002818BFFEF719FDE56349E043F659
:102A200030000096C4F20200416941F0200141618A
:102A3000416901F02001009100990096016841F080
:102A400040010160006801A900F04000009000987A
:102A50004FF4844001900220CDE902060320049047
:102A60000820059040F60000C4F2020000F58050F6
:102A7000FFF718FB46F22800C4F2020040F2E425FA
:102A800000F58F60C2F200054FF0206140224FF444
:102A9000806385E847002846C5E90436C5E906662F
:102AA000C5E90866FFF764FA002818BFFEF7CEFCF8
:102AB000A56305F13800046006B070BD80B590F8DC
:102AC0004230202B1CBF022080BD00294FF00103A3
:102AD00018BF002A01D1184680BD0023036301F00E
:102AE0000DFC0346184680BD80B501F089FB032824
:102AF00008BF80BD40F2981100EBC000C2F2000197
:102B000001EB8000C068002818BF804780BD00002E
:102B100080B501F075FB032808BF80BD40F2981115
:102B200000EBC000C2F2000101EB800080680028C9
:102B300018BF804780BD0000FEE7000010B52DEDF6
:102B4000088B88B3B0EE408A90ED010A90ED069AAA
:102B500090ED021A90ED07AA29EE000A38EE400A1D
:102B60002AEE011A30EE41BA04461BEE100A01F0BB
:102B70002DFC002808BFB0EE4B8A94ED030A94EDBB
:102B8000041A94ED052A20EE080A29EE011A30EE07
:102B9000010A2AEE021A30EE010A84ED068A84ED5B
:102BA000079ABDEC088B10BD9FED020ABDEC088BA7
:102BB00010BD00BF00000000002808BF704710B51E
:102BC000F5EE400A0446C0ED000A0020F1EE10FACE
:102BD000A061E0612EDD80EE200A9FED1E1A81EEDD
:102BE000000A04F037FB9FED1C1AB7EE002A20EE16
:102BF000011A31EE023A20EE000ABFEE005A30EE22
:102C0000033A30EE055A32EE411A80EE034A35EEB1
:102C1000055A30EE010A85EE035A80EE030A34EEBF
:102C2000041A84ED034A84ED041A84ED054A84ED08
:102C3000015A07E04FF07E519FED050AC4E90310E9
:102C40006061606084ED020ABDE81040704700BF1B
:102C500000000000DB0F4940F304B53F10B52DED37
:102C6000048B10B3B0EE408A90ED030A90ED041A85
:102C700090ED052A30EE010A30EE020A88EE009A45
:102C8000044619EE100A01F091FB00282046B0EE30
:102C9000480A08BFB0EE489A84ED069A84ED079A78
:102CA000FFF74CFFBDEC048B10BD9FED020ABDEC9D
:102CB000048B10BD00000000B0B5012802D9FF2030
:102CC00040B2B0BD40F20C25C2F20005044655F8F2
:102CD000200060B94820FDF725FF002845F82400B2
:102CE000EDD04821FDF7B7FB55F824000470002013
:102CF00040B2B0BD70B584B048B3067804463046E3
:102D000000F068F828B36188A1F201210A295FD890
:102D1000012202FA01F10A071DD111F0F00F30D0A3
:102D200040F2FF11009108218DF804100A300021B3
:102D30006A4600BF00EB41035B7802EB41056B7113
:102D400010F8113001310429AB71F3D131E0FE20CC
:102D50003BE0FC2039E04FF40071009108218DF830
:102D60000410023000216A4600EB41035B7802EB5D
:102D700041056B7110F8113001310429AB71F3D1A9
:102D800017E040F2FF21009108218DF80410123065
:102D900000216A4600EB41035B7802EB41056B7151
:102DA00010F8113001310329AB71F3D10020ADF8D7
:102DB0000B0030460121FDF769FE20786946FDF7DA
:102DC00051FE002818BF4FF0FF3040B204B070BD74
:102DD000FF20FAE701288FBF002040F20C21C2F249
:102DE000000151F82000704748B102280BD001289B
:102DF00014BF4FF6FF704FF4804000B2704742F2AC
:102E0000107000B2704747F2305000B270470000B7
:102E1000022905D2A0F2012189B2062909D805E0CC
:102E200007D1A0F2052189B2052902D8013840B2A4
:102E30007047FF2040B27047F0B581B008B3074635
:102E40000078FFF7C7FFE0B1014690F84400C0B139
:102E500001F11802002306E0012585B191F84450E4
:102E60000133AB420DD252F82340002CF4D06588D8
:102E70007E88B542F0D100252046002DEED101B06C
:102E8000F0BD002001B0F0BD022884BFB7EE000AFB
:102E9000704740B202A101EB800090ED000A70473C
:102EA00000001042000098410000803F70B538B12A
:102EB00004460078FFF700FF28B1FF2040B270BD44
:102EC000FE2040B270BD2078FFF784FF0028F4D0C8
:102ED00090F8442005469AB105F11800002104E05D
:102EE00095F84420013191420AD250F82120002A5D
:102EF000F6D0528863889A42F2D1FD2040B270BD6C
:102F00000A2ADAD85020FDF70DFE0028D5D0064653
:102F100020686168C6E9000106F118002821FDF764
:102F20009AFA62792078618886F828200322FDF7D2
:102F300073FC18B13046FDF7F1FDBEE795F844008B
:102F400005EB8001013085F84400002040B28E611D
:102F500070BD000080B59FED020A00F003F880BD4F
:102F60000000000070B52DED048B00283ED0054612
:102F70000078B0EE408AFFF72DFFC8B3B7EE000A25
:102F8000B4EE408AF1EE10FAC8BFB0EE408ABFEE50
:102F9000000AB4EE408A0446F1EE10FAB8BFB0EE73
:102FA000408A6879B1EE489A0028284608BFB0EEFA
:102FB000489AFFF741FFE8B12E7968883146FFF75C
:102FC00027FF002818D405463046FFF70DFF00EE16
:102FD000100AB8EEC00A29EE000ABDEEC00A10EED3
:102FE000100A04EB45014880002006E0FE2004E0C2
:102FF000FC2002E0FC2000E0FF2040B2BDEC048B8E
:1030000070BD00002DE9F04F87B0002852D0044673
:103010000078FFF7DFFE00284ED0054690F8440008
:1030200000284BD005F11806E8464FF0010A40F29F
:10303000E93B4FF0000908E00121002941D095F853
:10304000441009F1010989453AD256F82970002F38
:10305000F2D07A8861888A42EED1207842460023F5
:10306000FDF700FB70B1FDF761FDD7E90823801A79
:103070009941B0EB0B0071F1000016D300203876B7
:10308000FC2013E087F818A0FDF750FDC7E9080100
:103090003846414600F018F907F108030FCB07F155
:1030A0002C0C8CE80F00002000E0FF2000210029FC
:1030B000C5D106E0FE2004E0FC2002E0FC2000E098
:1030C000FC2040B207B0BDE8F08F000080B540F2B0
:1030D000342046F20041C2F20000C4F20001032293
:1030E000002380E80E0000F10C014FF4102C4FF487
:1030F000001E81E8085083618383FEF75FFC00288F
:1031000018BFFEF7A3F980BD80B540F25C2046F6FB
:103110000001C2F20000C4F200010322002380E893
:103120000E0000F10C014FF4102C4FF4001E81E84A
:10313000085083618383FEF741FC002818BFFEF727
:1031400085F980BD80B582B0002043F63001019042
:10315000C4F202010A6842F400120A600A6802F42A
:1031600000120192019A00900868002240F4800049
:1031700008600868052100F48000009000980C2089
:10318000FFF7DEF80C20FFF7D7F8452005210022D5
:10319000FFF7D6F84520FFF7CFF802B080BD00005A
:1031A00080B543F6FD5048F24C02C0F60000C0F670
:1031B0000002002101F06CFC40F23021C2F200015B
:1031C000086043F6057047F6E072C0F60000C0F6EE
:1031D0000002002101F05CFC80BD000081B00021F4
:1031E00043F630000091C4F20200026842F002028D
:1031F0000260026802F002020092009A00910268E6
:1032000042F040020260026802F040020092009A1E
:103210000091026842F001020260026802F00102BD
:103220000092009A0091026842F004020260026873
:1032300002F004020092009A0091016841F08001BE
:103240000160006800F080000090009801B07047B5
:1032500080B540F2443044F60001C2F20000C4F2EE
:10326000000148F2A06200234FF00C0CC0F20102F2
:1032700080E80E00C0E90333C0E905C3C361FFF76E
:103280003FFB002818BFFEF7E1F880BD80B540F293
:103290008C3041F20041C2F20000C4F2010100236F
:1032A0004FF00C0C4FF4E13280E80E00C0E903331C
:1032B000C0E905C3C361FFF723FB002818BFFEF771
:1032C000C5F880BDFEE700002DE9F0478846B1F85B
:1032D0000D10044608BA4FEA1049B8F811002679D3
:1032E000B8F80F1005BA304691FAB1FAFFF77CFD35
:1032F00007463046FFF7C8FD01EE109A9FED453AAC
:10330000B8EE412A9FED441A22EE032A22EE014A2A
:1033100002EE10AA15FB27F0B8EEC23A02EE100A30
:10332000A0799FED3E5AB8EEC22A22EE052A48B196
:10333000B4F84000A9EB0000B0F5805F0CDD4FF061
:10334000FF300DE00020A4F84090C4E9110084EDA6
:10335000024A84ED033A1CE010F5805F03DA012095
:10336000616C0844606494ED115A83EE003AB8EE43
:10337000C55A25EE015A34EE054A84EE004AA4F8F7
:10338000409020EE022A84ED033A84ED124A84ED47
:10339000024A94ED020A84ED042AB5EE400AF1EEE9
:1033A00010FA08DA30EE010AB5EE400AF1EE10FA32
:1033B000F8DB84ED020A94ED020AB4EE410AF1EE64
:1033C00010FA0ADB9FED162A30EE020AB4EE410A2B
:1033D000F1EE10FAF8DA84ED020A94F8280078B1D8
:1033E00031EE400A84ED020A94ED030A94ED041ACA
:1033F000B1EE400A84ED030AB1EE410A84ED040AFD
:1034000098F8130000EE100AB8EE400A84ED050AA1
:10341000BDE8F08700000039DB0FC94000008038AC
:10342000DB0FC9C0FEE7000000F0070080F00703D3
:10343000042B28BF04234FF0FF3C03380CFA03F39E
:1034400038BF0020994381400CFA00F022EA0000C6
:1034500008437047B0B52DED0A8B044610EE100AF4
:10346000B0EE618AB0EE419AB0EE60AAB0EE40BA1A
:1034700000F0A4FF002800F0A2801AEE100A00F06D
:103480009DFF002800F09B8019EE100A00F096FFC7
:10349000002800F0948018EE100A00F08FFF00283A
:1034A00000F08D806068B0EE4B0A90ED071AF0EEE8
:1034B0004A0AFDF7B3FD6068B0EE40BA90ED001A1D
:1034C00004F1280020EE01CA21EE0A0AFFF736FBBC
:1034D000207888B1012811D194ED051A94ED022AC3
:1034E00030EE411AB4EE428AF1EE10FAC8BFB0EEE7
:1034F000482A81EE029A01E09FED339A19EE100AF4
:1035000084ED04BA84ED050A00F058FF65689FED6C
:103510002E0A002808BFB0EE409A95ED032A95EDDB
:10352000010A95ED021A29EE022A94ED033A9FED65
:10353000279A2CEE084A2CEE000A34EE03BAB4EEB9
:10354000491A30EE42AA2BEE018AF1EE10FA84ED10
:10355000060A84ED078A84ED082A1ADD1BEE100A9C
:1035600000F02CFFA8B13AEE080A95ED051AB0EE6E
:10357000C00AB4EE410AF1EE10FA0ADC95ED040A35
:10358000B0EECB1AB4EE401AF1EE10FAD8BF84EDCB
:1035900003BA3AEE088A18EE100A00F00FFF70B175
:1035A000D5ED050AF4EE490AF1EE10FA05DDB0EEAC
:1035B000480AFCF7C3FFB0EE408A84ED098A94ED17
:1035C000090ABDEC0A8BB0BD00000000BD3786358E
:1035D00070B52DED048B90B3044650681646B0EEDE
:1035E000408A0D4600F0EAFE58B3B06800F0E6FEEF
:1035F00048B3F06800F0E2FE38B3306900F0DEFE58
:1036000028B3706900F0DAFE18B3B7EE000A80EE56
:10361000089A666019EE100A00F0D0FED8B1D6ED17
:10362000060A04F12800B0EE480A84ED029AFFF77A
:10363000C3FA2046257000F013F800200CE0FF20AC
:103640000AE0FF2008E0FF2006E0FF2004E0FF2062
:1036500002E0FF2000E0FF2040B2BDEC048B70BD13
:1036600010B558B100249FED070AC0E90344446136
:1036700044622830FFF7F2FA60B210BDFF2460B256
:1036800010BD00BF0000000000280EBFFF21002178
:10369000C16048B270470000000000000000000058
:1036A000EFF30980BFF36F8F154B1A681EF0100FF0
:1036B00008BF20ED108A20E9F04F10602DE90900C5
:1036C0004FF0500080F31188BFF34F8FBFF36F8F1F
:1036D00002F03EFB4FF0000080F31188BDE80900C6
:1036E00019680868B0E8F04F1EF0100F08BFB0EC82
:1036F000108A80F30988BFF36F8F704700BF00BF47
:10370000D0040020000000000000000000000000C5
:10371000074B19680868B0E8F04F80F30988BFF3D9
:103720006F8F4FF0000080F31188704700BF00BF1B
:10373000D004002080B500F07BFE80BD90ED000A33
:1037400091ED001AB7EE002A30EE011AB4EE421ADB
:10375000F1EE10FAD8BF704782EE011A20EE010A8E
:1037600080ED000A91ED000A21EE000A81ED000AC9
:103770007047000030B390F870201AB3436990EDA1
:10378000010A90ED1B1A93ED012A30EE411AB4EEB6
:10379000421AF1EE10FA28DB897831B380ED1B0A6A
:1037A00093ED000A90ED291A9FED122A30EE010ADE
:1037B000B4EE420AF1EE10FA80ED290A05DD9FED24
:1037C0000C1A0BE0FF2040B270479FED0C1AB4EECC
:1037D000410AF1EE10FA05DA9FED071A30EE010A00
:1037E00080ED290A511E80F87010002040B2704709
:1037F000DB0FC9C0DB0F4940DB0FC940DB0F49C0FD
:103800002DE9F04F81B02DED048B82B08246002867
:103810004FF0FF0000F0E0818946002900F0DC81D4
:10382000FDF784F904F037FB9FEDF68A00EE100AED
:1038300080EE080A8AED010AFDF778F9DAE9022339
:10384000801A994104F027FB00EE100A80EE080A66
:103850008AED040AFDF76AF999F8002040F2DA359A
:10386000002AC2F20005CAE902018AF8002000F02D
:10387000A4809AF81800002800F0AE80022800F01A
:103880001781012840F09C819FEDDF9A9FEDDF8A30
:1038900000276FF047084FF426750A26CDF80490EC
:1038A0009AED280A0AEB070480EE090A0AEB0809D8
:1038B000DAED041AD4ED170A09F1F000B0EE481A57
:1038C000FFF7C8FD84ED1D0ADAED041A9AED190A16
:1038D000D4ED170A09F5C070B0EE481A04F1740B64
:1038E000FFF7B8FD04F17C01584684ED1F0AFFF78D
:1038F00025FF94ED1D0A0AEB050084ED210AFFF770
:103900001DF9DAF8140084ED230A3044FFF72AFB8E
:10391000043708F148082035042F06F10806BFD007
:103920009FEDBA8ADAED041ADAED160A9AED290A41
:103930000AF5E470B0EE481AFFF78CFDDAED041AD0
:10394000DAED1A0A0AF50470B0EE481A8AED250A73
:10395000FFF780FD0AF53E708AED260AFFF7EEF8C4
:10396000DAF814008AED270A1A30FFF7FBFADDF8BF
:10397000049099F80100002800F0358140F2DA3512
:10398000C2F200052878002840F01D8199F8020055
:10399000002800F01881504600F0B0F9504600F0C1
:1039A00019FADAF814009AF87020007A022110440B
:1039B0008AF818108AF8700005E10A24DAF8140071
:1039C0002044FFF7C7FA0834122CF7D0DAF81400B5
:1039D0001A30FFF7BFFAF6E09FED8C8A4FF4267499
:1039E0004FF0A80B6FF003080A2500BF0AEB0B0687
:1039F0003046FFF749FE0AEB0807D7ED180ADAED63
:103A0000041A3046B0EE480AB0EE481AFFF722FD1D
:103A10000AEB040087ED1E0A87ED220AFFF78EF8F5
:103A2000DAF8140087ED240A2844FFF79BFA2034C3
:103A30000BF1480B08F10408B4F52E7F05F10805D9
:103A4000D4D09FED728ADAED041ADAED160A9AEDF7
:103A5000290A0AF5E470B0EE481AFFF7FBFCDAED2C
:103A6000041ADAED1A0A0AF50470B0EE481A8AED63
:103A7000250AFFF7EFFC0AF53E708AED260AFFF7EC
:103A80005DF8DAF814008AED270A1A30FFF76AFAAF
:103A900099F8010040F2DA350028C2F2000500F082
:103AA0009280504600F02AF9504600F071F982E009
:103AB00050464946CDF80490FFF75CFE9FED529AC0
:103AC0009FED528A00276FF047094FF426750A26AA
:103AD0009AED280A0AEB070880EE090A0AEB0904A6
:103AE000DAED041AD8ED170A04F1F000B0EE481A26
:103AF000FFF7B0FC88ED1D0ADAED041A9AED190AF9
:103B0000D8ED170A04F5C070B0EE481A08F1740B2E
:103B1000FFF7A0FC08F17C01584688ED1F0AFFF76B
:103B20000DFE98ED1D0A0AEB050088ED210AFFF74E
:103B300005F8DAF8140088ED230A3044FFF712FA8A
:103B4000043709F148092035042F06F10806BFD0D3
:103B50009FED2E8ADAED041ADAED160A9AED290A9B
:103B60000AF5E470B0EE481AFFF774FCDAED041AB7
:103B7000DAED1A0A0AF50470B0EE481A8AED250A41
:103B8000FFF768FC0AF53E708AED260AFEF7D6FFBD
:103B9000DAF814008AED270A1A30FFF7E3F9DDF8A6
:103BA000049040F2DA3599F80200C2F2000550B9EB
:103BB000504600F0A3F8504600F00CF9012000E058
:103BC00000208AF81800DAF814000A30FFF792F89B
:103BD00099F802002870002040B202B0BDEC048BBE
:103BE00001B0BDE8F08F504600F088F8504600F074
:103BF000F1F8002040F2DA358AF81800C2F2000528
:103C0000E1E700BF0024744900C0DA45000000006D
:103C10002DE9F0472DED028B044600284FF0FF0000
:103C200066D08846002963D0B5EE400AB0EE408ADF
:103C3000F1EE10FA5CDDC4F81480FCF753FD08F1D6
:103C4000240908F10A0A04F1A80704F516750026EC
:103C50000AEB0600FFF72AF938460121B0EE480AC0
:103C60004A46FFF7B5FC6069B0EE480AD0ED290A74
:103C70002846FEF7A1FF6069B0EE480AD0ED2A0A97
:103C800005F14000FEF798FF08364837082E05F189
:103C90002005DDD008F11A00FFF708F904F5E470FB
:103CA00008F164020121B0EE480AFFF791FC04F527
:103CB000047008F184020121B0EE480AFFF788FC85
:103CC0006069B0EE480AD0ED2B0A04F53670FEF7B5
:103CD00073FF6069B0EE480AD0ED2C0A04F53E701F
:103CE000FEF76AFF04F16C003421FCF7B4FB0020FE
:103CF00040B2BDEC028BBDE8F0870000002841D047
:103D0000F0B581B02DED028B9FED208A044600F1C5
:103D1000A8056FF01F0600BF2846FFF7A1FC05F1BC
:103D20009000FFF79DFCA71907F51E70B0EE480A3A
:103D3000FEF794FF07F52E70B0EE480AFEF78EFFEF
:103D4000203605F14805E7D004F5E470FFF788FC5C
:103D500004F50470FFF784FC9FED0C8A04F53670BF
:103D6000B0EE480AFEF77AFF04F53E70B0EE480A5E
:103D7000FEF774FF0020BDEC028B01B0BDE8F040FF
:103D800040B27047FF2040B2704700BF0000000003
:103D9000E0B170B504466FF0470500BF661906F143
:103DA000F000FFF771FC06F5C070FFF76DFC4835B9
:103DB000F4D004F5E470FFF767FC04F50470FFF736
:103DC00063FC0020BDE8704040B27047FF2040B265
:103DD0007047000070B10021C0E91D11C0E91F113A
:103DE000C0E92111C0E92311C0E92511C0F89C10D8
:103DF00048B27047FF2148B27047000080B500F01C
:103E000043FE00F09FFE80BDB0B501380024B4EB46
:103E1000106F1CBF0120B0BD4EF21005CEF20005A0
:103E200068604FF0FF300F2100F0F0FA0720AC601F
:103E300028602046B0BD000080B5FEF707FA02F00A
:103E400089FE012818BF02F05BF880BD70B592B002
:103E500006AC20463021FCF7FEFA002543F6400070
:103E60000595CDE90355CDE901550095C4F2020051
:103E70000168022641F080510160006800F0805026
:103E80000090009847F200000095C4F2000001681D
:103E900041F480410160006800F480400090009887
:103EA000012006904FF4803007904FF480000D9071
:103EB00006200E90A820CDE90F0604201190204680
:103EC0000C96FEF75FFB88B90F20CDE901064FF491
:103ED000A05004904FF48050059001A8052103954F
:103EE000FEF742FA002804BF12B070BDFDF7AEFA2B
:103EF0004EF68850CEF20000016841F47001016076
:103F00007047000010B500F05DFB44F2010048F27C
:103F10002802C0F60000C0F60002002100F0B8FD43
:103F200040F6DC44C2F20004206043F6697048F2B7
:103F30000402C0F60000C0F60002002100F0A8FD57
:103F4000606002200A21002200F0D2FBA060032062
:103F50002821002200F0CCFBE06000F063FB00F0C1
:103F600093FD00F0EFFD10BD00F014FB03F05FFDCA
:103F70009FED210B53EC102B03F0D2FB03F02AFD35
:103F80000446002000F0D2FA00F0FAFA40F2E018FD
:103F9000C2F2000805464046FDF764F840F21429D5
:103FA000C2F200094846FDF7C7F92F1940F6681517
:103FB00040F6DC46C2F20005C2F200060AE000BF8D
:103FC000F06829460022002300F0E2FB384600F0AA
:103FD000BDFA27440A20FDF7BDF90028F0D0484675
:103FE0004146FDF763F840462946FCF725FE484662
:103FF000FDF7A2F9E4E700BF0000000000407F40A9
:1040000000F0C8FA03F013FD9FED230B53EC102BC7
:1040100003F086FB03F0DEFC8046002000F086FA09
:1040200000F0AEFA0446FDF717F840F69015C2F21C
:1040300000059FED1B0A01462846FFF7E9FD04EB4A
:10404000080640F6DC4940F6B44740F6B044C2F2F8
:104050000009C2F20007C2F2000400BFD9F80C0048
:1040600039460022002300F0FFFA387897F8241030
:1040700097F82520207028466170A270FCF7ECFEAE
:1040800028462146FFF7BCFB304600F05FFA464465
:10409000E4E700BF00BF00BF0000000000407F4019
:1040A0000000FA4310B5846B2068406994F8411011
:1040B000212907D110F0800004D00020E0842046A0
:1040C00000F090F82068406994F84210222907D146
:1040D00010F0400004D00020E085204600F05AF89F
:1040E000606C40F0100060642046FEF7F5FB10BDE8
:1040F00080B50168806B0968C9052FD40021C1858E
:10410000016851E8031F026821F4807142E803133B
:10411000002BF5D1016851E8051F026821F001016B
:1041200042E80513002BF5D1016851E8051F02682C
:1041300021F0400142E80513002BF5D1202180F841
:104140004210016B012909D1016851E8031F02687F
:1041500021F0100142E80313002BF5D10021416347
:10416000016B012903D1818DFEF7B4FB80BDFEF701
:10417000BBFC80BD80B5806B01214163016B0129CF
:1041800004D1818D4908FEF7A5FB80BDFEF7C0FC78
:1041900080BD0000016851E8031F026821F490719E
:1041A00042E80313002BF5D1016851E8051F0268AE
:1041B00021F0010142E80513002BF5D1016B012923
:1041C0000AD100BF016851E8031F026821F0100105
:1041D00042E80313002BF5D1202180F84210002182
:1041E00001637047016851E8031F026821F0C001B4
:1041F00042E80313002BF5D1202180F841107047CD
:1042000044F600010068C4F2000101F54C420323AA
:10421000904208BF0123401A18BF1846704700009B
:1042200010B504460068D4E902C22369016921F48B
:10423000405111430161626943EA0C01E369114392
:10424000C268194349F20C639A431143C160416942
:10425000A26921F4407141F20043114340F48062AD
:10426000C4F201039A42416102D1FEF745F901E02F
:10427000FEF730F9E16963681922B1F5004FA0FB40
:1042800002011CD15A00DB0FFBF7EEFF48F21F5171
:10429000C5F2EB11A0FB01235A096FF0630302FB87
:1042A0000300322303EBC000A0FB01014FF4F870C0
:1042B00000EA111000EB0210C1F342111AE09A005B
:1042C0009B0FFBF7D1FF48F21F51C5F2EB11A0FB8A
:1042D00001235A096FF0630302FB0300322303EB4F
:1042E0000010A0FB0101F02000EA511000EB0210C9
:1042F000C1F3431122680843906010BDF0B581B04E
:10430000134600270446816283854764222084F88F
:104310004200E06B44F2F10544F275160A4621684A
:10432000C0F60005C0F60006C0E90F5644F2A50627
:10433000C0F600060431C0E91367FDF781FE38B10D
:1043400010206064202084F84200012001B0F0BDFC
:1043500000972068016800914068009000982069EB
:1043600050B100BF206850E8030F216840F480700E
:1043700041E80302002AF5D1206850E8050F2168C2
:1043800040F0010041E80502002AF5D1206850E81C
:10439000050F216840F0400041E80502002AF5D1F0
:1043A000002001B0F0BD0000FEE7000000F0FF407B
:1043B000B0F1FF4018BF01207047000000F0FF403F
:1043C000B0F1FF4018BF01207047000020F000400E
:1043D000A0F1FF40B0FA80F040097047002848BFC4
:1043E000704700F01F01012202FA01F14EF20012A3
:1043F0004009CEF2000242F8201070474EF60C50F1
:10440000CEF200000068C0F3022070474EF614534D
:1044100000F00F02CEF2000309011A4400F16043DC
:10442000B0F1FF3FC8BF03F5644211707047000050
:104430004EF61F50CEF200000021017070470000C0
:104440004EF60C51CEF200010A684FF6FF031A40F7
:1044500060F30A2242F0806040F0FD70086070470F
:10446000F0B581B0F0B1044640F2D040C2F2000095
:104470000068A0421FD001F08BF940F2D840C2F290
:1044800000006569076840F2E040C2F2000006687B
:1044900001F0A2F9BD424FF0020018BFB5420DD1A4
:1044A00001B0F0BD4FF0500080F31188BFF36F8F63
:1044B000BFF34F8FFEE7002001B0F0BD45F2C00012
:1044C000C2F2000085420CD045F2D4010120C2F2B4
:1044D0000001002D08BF04208D4208BF042001B058
:1044E000F0BDA06A10B1022001B0F0BD94F85810E0
:1044F0000320012908BF022001B0F0BDFDF7B4FE82
:10450000FFF7A4FCFEF76AFEFEF71CFEFEF7DEFDD9
:10451000FEF7FAFDFEF79CFEFEF7B8FE00F03EF84F
:10452000FEF73EFE00F064F8FEE70000EFF30581C1
:1045300000291CBF6FF005007047002804BF002051
:10454000704780B501F028FA002080BD10B582B018
:10455000EFF3058119B16FF0050002B010BD0446FC
:1045600002F00CFB211A0129019005DB01A801F0E2
:104570003DFA002002B010BD6FF0030002B010BD84
:1045800080B5EFF3058010B102F0FEFA80BD02F0B5
:10459000F5FA80BD4FF47A7070470000EFF30580A4
:1045A00000281CBF6FF00500704740F29410C2F263
:1045B00000000168002911BF4FF0FF3001210160A8
:1045C0000020704780B5EFF3058000281CBF6FF016
:1045D000050080BD02F0BEFA28B1022805D101F025
:1045E000AFFB002080BD012080BD4FF0FF3080BDBB
:1045F00010B5EFF3058000281CBF6FF0050010BD5B
:1046000040F29414C2F20004206801281CBF4FF04D
:10461000FF3010BDFFF78EF80220206001F03EFB56
:10462000002010BD10B5EFF3058018B16FF0050440
:10463000204610BD02F08EFA02280ED080B902F09A
:104640007BFC01284FF001040CD002F083FA002813
:1046500008BF4FF0FF34204610BD0024204610BD97
:104660004FF0FF34204610BD10B582B01C46B0FAA2
:1046700080F3B1FA81F25B095209EFF3058CBCF1CA
:10468000000F42EA030219D0002C18BF0124224374
:1046900015D10022019201AA01F036FF01281AD19A
:1046A0000198A8B14EF60450CEF200004FF08051B0
:1046B0000160BFF34F8FBFF36F8F09E01AB16FF046
:1046C000030002B010BD224601F05CFE012806D1B5
:1046D000002002B010BD6FF0020002B010BD6FF0FC
:1046E0000100002C08BF6FF0020002B010BD0000F6
:1046F000B0B582B0144600294FF00005EFF30582F3
:1047000018BF002802D1284602B0B0BD002AFAD155
:104710009CB1A568D5B1E268502A16D32269A2B12E
:10472000D4F814C001FB00F2002394454FF00002BE
:1047300028BF012210D24DB10EE0012300226AB938
:10474000E3B1002201F012FC0EE01DB9E2680AB9E3
:104750002269C2B100220023002AF1D0A368226995
:104760000025009501F026FC054655B1002C14BF2C
:1047700021680021284601F0D9F8C4E70025002D62
:10478000F4D10025BFE76269B2FA82F25309D5E796
:10479000B0B582B01C46B0FA80F3B1FA81F5EFF300
:1047A00005825B096D09002A43EA050207D0002C47
:1047B00018BF0124224306D06FF003052CE0CAB1D4
:1047C0006FF0030528E00022019201AA002301F006
:1047D0004FFD01281CD10198E8B14EF60450CEF2ED
:1047E00000004FF080510160BFF34F8FBFF36F8F18
:1047F000002511E022460023002501F067FC012876
:104800000AD06FF00105002C08BF6FF0020503E02D
:104810006FF0020500E00025284602B0B0BD0000A0
:1048200010B50C46EFF3058100291CBF6FF00500A1
:1048300010BD014620F0010050B111F001010AD174
:10484000214601F0B7FE012804BF002010BD09E099
:104850006FF0030010BD214601F090FF012804BF56
:10486000002010BD6FF00100002C08BF6FF00200A7
:1048700010BD000070B5EFF30581B9B900280446FA
:1048800014BF60680020010710D494B1A36843B13D
:10489000E26800214F2A4FF0000288BF01220AD8A7
:1048A0004BB9E168B1FA81F1490903E000252846D6
:1048B00070BD0121002200F001063AB1A168002E6E
:1048C0000CBF0120042001F03FFB06E0C9B1002E1F
:1048D0000CBF0120042001F02BFB054635B1002C54
:1048E00014BF21680021284601F020F8B5FA85F0B0
:1048F000400986F00101084308BF45F0010528463C
:1049000070BD0025002DEAD1F0E7000080B5EFF37F
:10491000058100291CBF6FF0050080BD014620F015
:10492000010040B111F0010108D100210022002353
:1049300001F0CCFB04E06FF0030080BD01F000FD4E
:10494000013818BF6FF0020080BD0000B0B584B020
:1049500048B3B1F1FF3F26DD04464FF0FF3003902E
:10496000EFF3058018B300250DF1080C2046012255
:1049700000230295CDF800C002F050F803AB2046AA
:1049800000210022009502F049F80298D0B14EF6BD
:104990000450CEF200004FF080510160BFF34F8F02
:1049A000BFF36F8F0EE06FF0030003900AE0204624
:1049B0000122002301F0B4FF03AB204600210022B6
:1049C00001F0AEFF039804B0B0BD00002DE9F04F38
:1049D00083B00C46EFF3058129B16FF00507384627
:1049E00003B0BDE8F08F0546002849D44FF0000B16
:1049F0009246A00758BFAB4602F0C0F800906FF097
:104A0000010804F0010054460027BAF1000F08BF66
:104A10006FF00208019002E04746002EDFD0002030
:104A2000594602AA234602F063F906460128F3D14B
:104A3000029807EA050140EA01090198002809EAFD
:104A4000050007D100286FF0020718BF4F4607D0B6
:104A5000C5E700BFA8426FF0020708BF4F46BED0AF
:104A6000BAF1000FBBD002F089F800994F46401A06
:104A7000241A4FF0000038BF0446002ECFD1AEE715
:104A80006FF00307ABE7000080B502F05DF880BD72
:104A900070B584B08E46002100280391EFF30581A4
:104AA00046D0002944D1FAB19369002B08BF1823DE
:104AB000382B16D81179C90713D155699468116834
:104AC0004FEA950C002D08BF4FF0800CFCB1D66862
:104AD0005C2E1BD3D5B11569C5B10024012555B98C
:104AE0001BE0002004B070BD0124002118234FF00A
:104AF000800C00258DB1946812690294CDE90032D2
:104B00006246734601F0D0FE039011E00CB9D46800
:104B10009CB100250024002DEDD14CB103AC0093D5
:104B20001FFA8CF27346019401F08AFE012802D12B
:104B3000039804B070BD0020E6E71469B4FA84F469
:104B40006409D6E710B5EFF3058100291CBF6FF0AB
:104B5000050010BD044660B12046FFF781FC042823
:104B600004BF6FF0020010BD204600F093FF00204C
:104B700010BD6FF0030010BDF0B581B00D4645F2D9
:104B8000E80140F2D046C2F20001C2F200060F680E
:104B900031680446081D00F087FD601C0AD14DB144
:104BA0003068011D45F2C000C2F2000000F0D8FDDF
:104BB00001B0F0BD3068E41944600AD340F2E0402F
:104BC000C2F2000000683168043100F0ABFD01B0B2
:104BD000F0BD40F2D840C2F20000006831680431F4
:104BE00000F0A0FD45F24C00C2F2000001688C42CA
:104BF00038BF046001B0F0BD70B5044600F0C8FDD8
:104C000044F62010C2F20000016840F2D0450131A4
:104C10000160C2F20005296845F2B406C2F200063E
:104C200041B1306860B92868E16AC06A884298BFBB
:104C30002C6005E02C600068012801D100F0DEF94D
:104C400044F62C10C2F20000016801310160616479
:104C500044F63011C2F20001E06A0A68904288BF4F
:104C6000086040F2E84100EB8000C2F2000101EB75
:104C70008000211D00F074FD00F0AEFD306880B1B1
:104C80002868E16AC06A884228BF70BD4EF60450A9
:104C9000CEF200004FF080510160BFF34F8FBFF3A1
:104CA0006F8F70BD70B582B000F072FD45F2EC06FA
:104CB000C2F20006306850BB44F6EC74C2F2000445
:104CC000204600F01FFD45F20005C2F2000528460F
:104CD00000F018FD40F2D440C2F20000046040F23F
:104CE000E440C2F2000040F2DB3240F27C43056057
:104CF0000025C2F20002C2F200030A201021009532
:104D000001F058F9306010B103A100F00FFE00F07F
:104D100063FD02B070BD00BF546D72510000000011
:104D2000F0B581B044F62415C2F200052868E0B160
:104D300045F2D40644F62017C2F20006C2F200077C
:104D400000F026FDF068C468201D00F0ADFC386856
:104D50000138386028680138286000F03DFD2046A1
:104D600000F058F828680028EAD101B0F0BD000032
:104D700080B5026C002A08BF80BDD0E902C313448D
:104D8000C360634524BF0368C360C368084619460F
:104D9000FBF7E2FA80BD000070B5866B036C044639
:104DA000E3B115461AB3E0681A46FBF7D5FAE16895
:104DB000206C2268091A9142E16003D2A168404246
:104DC0000844E060A81EB0FA80F040093146002E89
:104DD00018BF01210840361A002516E0206800257A
:104DE00098B9A06801F0CCFFA56005460DE06068A9
:104DF0001A46FBF7B1FA216CD4E9010200250844F8
:104E00006060904224BF20686060711C2846A163E6
:104E100070BD000010B5044690F85900022808BF84
:104E200010BD012803D030B9206B00F0EDFC204606
:104E300000F0EAFC10BD4FF0500080F31188BFF382
:104E40006F8FBFF34F8F00BFFEE70000416A00295C
:104E50000FBF0020006B0068C0F1380070470000F1
:104E600040F2D441C2F2000109680A68B2FA82F342
:104E70005B090360002A0EBF0020C8680068704705
:104E800040F61450C2F20000C21D22F0070210F0DA
:104E9000070CA0EB020318BF104645F2B802C2F29D
:104EA00000020021C2E900014FF47052BCF1000F72
:104EB00018BF03F570520244083A40F2DC4322F076
:104EC0000702C2F200031A60C2E90011111A1A683F
:104ED000C0E9002145F24800C2F20000016045F23D
:104EE0004000C2F20000016045F21400C2F200006E
:104EF000012101707047000040F2E8444EF604556D
:104F0000C2F20004CEF200054FF08056FFF708FF12
:104F100020680228FAD32E60BFF34F8FBFF36F8F44
:104F2000F4E70000002808BF704780B50021016049
:104F3000C0E9021100210022002301F0C7F8BDE8FA
:104F400080407047B0B5049D002914BF2A602D60D1
:104F5000C5E90F01284601211C4601F077F885F8C4
:104F60004C40B0BD2DE9F0470A9C8246206B1646A6
:104F70000F46DDE908599100A5229846FBF763FA30
:104F8000206B00EB8600A0F1040020F007067FB143
:104F900004F13400002100BF7A5C42547A5C1AB1FB
:104FA0000F2901F10101F7D3002084F8430002E04A
:104FB000002084F834000027201D372D28BF372516
:104FC000E562C4E9135700F0A9FB04F1180000F0F2
:104FD000A5FBC5F13800A061304651464246246128
:104FE0006462676584F8587000F04AFBB9F1000FFD
:104FF000206018BFC9F80040BDE8F087B0B540F2A6
:10500000E8450024C2F20005281900F07BFB1434A7
:10501000B4F58C6FF8D145F21804C2F200042046B2
:1050200000F070FB45F22C05C2F20005284600F0A6
:1050300069FB45F26000C2F2000000F063FB45F23C
:10504000D400C2F2000000F05DFB45F2C000C2F2E5
:10505000000000F057FB40F2D840C2F200000460AC
:1050600040F2E040C2F200000560B0BD80B545F2FC
:10507000B802C2F2000200BF114612688242FBD39E
:10508000D1F804C001EB0C03834203D140686044B3
:1050900048600846D0F804C000EB0C03934201D0EE
:1050A00013460BE040F2DC43C2F200031B689A4255
:1050B00004D0D2E9003E0EEB0C0242608142036054
:1050C00018BF086080BD000080B58C46014641F8DD
:1050D00004CF9445006108D99A4201D29C4511D26F
:1050E00040F2D440C2F2000007E08069D21A824246
:1050F00008D240F2E440C2F20000006800F012FB67
:10510000002080BD012080BD10B5044600F040FBAA
:10511000A06BB0FA80F0440900F05EFB204610BDA1
:1051200010B5044600F034FBA06BE16B401AB0FAF6
:1051300080F0440900F050FB204610BD084800688C
:10514000006880F308884FF0000080F3148862B68E
:1051500061B6BFF34F8FBFF36F8F00DF00BF00BF9B
:1051600008ED00E070B582B040F2D442C2F2000215
:1051700012680546D2680E46D468201D00F094FAE5
:1051800094F82800410704D400F0FE0084F82800B9
:1051900010E0A0693246411920462B46FFF794FFE4
:1051A00040B10026204600212A460023009601F047
:1051B00087FF20B1216A2046884702B070BD4FF0BA
:1051C000500080F31188BFF36F8FBFF34F8F00BF84
:1051D000FEE700002DE9F04186B045F2EC07C2F28F
:1051E0000007386802A900224FF0000801F0CAF851
:1051F00000286AD001AC02AD0BE000F0FE0086F89A
:10520000280000BF38682946002201F0BBF80028BA
:105210005BD00298B0F1FF3F03DCDDE90320059984
:10522000904702980028EDD4049E706910B1301D9B
:1052300000F03AFA204600F0B3F802990929E1D8C3
:105240000246DFE801F0080808052A390808052A9F
:1052500096F82800D1E796F82800039BB16940F042
:10526000010086F8280019443046FFF72DFF00287A
:10527000C8D0316A3046884796F828004007C1D523
:105280000398B16900230A1830460021CDF8008048
:1052900001F016FF0028B5D123E096F8280040F071
:1052A0000101039886F82810B06188B18118304652
:1052B0001346FFF709FFA5E796F8280081073FF599
:1052C0009CAF304600F0A0FA9CE706B0BDE8F08144
:1052D0004FF0500080F31188BFF36F8FBFF34F8FF3
:1052E000FEE74FF0500080F31188BFF36F8FBFF3DC
:1052F0004F8F00BFFEE7000070B582B00E46044637
:1053000000F01EFD01A800F04BF8019919B101F061
:1053100013FE02B070BD05464EB9A54207D301F099
:105320000BFE20462946FFF71DFF02B070BD4EB1AF
:1053300040F2E440C2F2000000680068B0FA80F079
:10534000420900E0002245F2EC00C2F200000068D1
:10535000611B00F0FFFA01F0EFFD0028D9D14EF6F5
:105360000450CEF200004FF080510160BFF34F8F28
:10537000BFF36F8F02B070BD40F2D840C2F20000A0
:105380000168096821B10068C068C068406801E030
:105390004FF0FF3045F24C01C2F200010860704747
:1053A00070B5044601F0EAFB40F2CC46C2F20006BA
:1053B00031680546884203D200F008F8012000E079
:1053C000002020602846356070BD00002DE9F041C6
:1053D00082B040F2D447C2F200073868016891B346
:1053E0004FF0000809E000BF60603868294624617A
:1053F00000F098F93868016829B3C068C468066885
:10540000251D284600F050F9216A2046884794F867
:1054100028004007EED5A0693044B042E4D82046C9
:10542000002132460023CDF8008001F049FE00281B
:10543000E0D14FF0500080F31188BFF36F8FBFF3BE
:105440004F8F00BFFEE740F2E441C2F200010A685C
:1054500008603A6002B0BDE8F081000081B0002031
:10546000009040F2C000C2F2000000684FF050010E
:1054700081F31188BFF36F8FBFF34F8F013001D0DD
:10548000FEE700BF00980028FCD001B07047000084
:1054900082B001AC2046FFF7E3FC0199FFF72CFF37
:1054A000FFF798FEF6E70000F0B581B0044600F083
:1054B0006FF994F94560012E0FDB04F1240500BF5C
:1054C000286850B1284601F0EFFC002818BF00F012
:1054D00051FB70B2013E0128F2DCFF2684F84560E2
:1054E00000F07AF900F054F994F94470012F0EDBC2
:1054F00004F11005286850B1284601F0D5FC0028B9
:1055000018BF00F037FB78B2013F0128F2DC84F8C5
:10551000446000F061F901B0F0BD00002DE9F043F6
:1055200081B0044600F00CFC40F2DC46C2F20006FA
:105530003068002808BFFFF7A3FC45F21408C2F248
:10554000000898F80000002818BF4FF000402042E3
:105550000DD0002401F0F0FC60071ED04FF0500089
:1055600080F31188BFF36F8FBFF34F8FFEE7C4B195
:1055700014F0070004F108011EBF081A00F1080129
:105580005FEA41700ED04FF0500080F31188BFF3F6
:105590006F8FBFF34F8F00BFFEE7204601B0BDE81D
:1055A000F083002145F24009C2F20009D9F8000059
:1055B0004A1E8242CDD245F2B800C2F20000056810
:1055C0002F4657F8042F8A4211D22B685BB100BFD7
:1055D0001F4657F8042F28461D468A4207D22B68DB
:1055E000002BF5D103E045F2B800C2F200003368A9
:1055F0009D42AED004682B68521A112A036010D362
:105600006818430709D04FF0500080F31188BFF3AA
:105610006F8FBFF34F8F00BFFEE742603960FFF727
:1056200025FD45F248003968D9F80020C2F2000093
:105630000368511A9942C9F8001038BF016098F800
:105640000000396800284FF0000018BF41F0004109
:10565000286045F25400C2F2000002680834396044
:10566000511C016076E7000040F2D040C2F2000019
:10567000016819B101680A6D01320A650068704756
:10568000034645F25D40C0F600004FF0807C21F0FB
:10569000010103E903106FF0020043F8240CA3F1A9
:1056A000440043F8202C7047D0E9013201699A6028
:1056B000D1F804C082688445536008BF4A60002264
:1056C00002610868013808600868704744F634339E
:1056D000C2F20003036044F63410C2F20000086016
:1056E000802010607047000044F69073C2F20003FF
:1056F000036044F69030C2F2000008604FF48070FE
:10570000106070474FF0FF31024642F8081F002139
:105710004260C0E90322016070470000002101617E
:105720007047000080B5D1F800C01CF1010207D01D
:1057300000F108039E465B681A686245FAD901E0E9
:10574000D0F810E0DEF8042008614A609160C1F8EA
:1057500008E0CEF8041001680131016080BD00004E
:10576000D0F800C0436808619A684B608A609A6804
:10577000996051600CF1010101607047DFF80C0085
:10578000016841F470010160704700BF88ED00E0DE
:105790004FF0500080F31188BFF36F8FBFF34F8F2E
:1057A00040F2C000C2F2000001684A1C026001B170
:1057B00070474EF60450CEF200000068000608BFA5
:1057C00070474FF0500080F31188BFF36F8FBFF325
:1057D0004F8F00BFFEE7000040F2C000C2F20000A1
:1057E000016839B10139016018BF7047002080F3AA
:1057F000118870474FF0500080F31188BFF36F8F0E
:10580000BFF34F8FFEE70000B0B5002808BFB0BD62
:10581000044645F21400C2F20000007854F8041C5B
:10582000002818BF4FF0004008420CD0A4F1080532
:105830002A6892B14FF0500080F31188BFF36F8F48
:10584000BFF34F8FFEE74FF0500080F31188BFF396
:105850006F8FBFF34F8F00BFFEE721EA000044F8CF
:10586000040C00F06DFA45F24001C2F2000154F858
:10587000040C0A68104408602846FFF7F7FB45F25D
:105880005800C2F2000001680131016001F054FBD0
:10589000B0BD00004EF21000CEF200000021016009
:1058A000816040F20001C2F20001096844F6D3525F
:1058B000C1F26202A1FB02124FF0FF3101EB921123
:1058C0004160072101607047EFF30580102814D371
:1058D0004EF2F031CEF20001405C44F61411C2F2F7
:1058E00000010978884208D24FF0500080F31188F7
:1058F000BFF36F8FBFF34F8FFEE74EF60C50CEF223
:10590000000044F618110068C2F20001096800F4B2
:10591000E060884298BF70474FF0500080F31188D4
:10592000BFF36F8FBFF34F8FFEE7000045F2740C9B
:105930000022C2F2000C00BF5CF8323023B1013209
:10594000082A08BF7047F7E70CEBC2034CF8321087
:105950005860704770B515460E460446FFF718FFAD
:1059600094F84400FF2804BF002084F8440094F811
:105970004500FF2804BF002084F84500FFF72CFFF6
:10598000A06B28B904F1240031462A4600F014F92E
:105990002046FFF789FD70BD10B5D8B1044644F626
:1059A0002810C2F20000006848B14FF0500080F3A8
:1059B0001188BFF36F8FBFF34F8F00BFFEE700F07A
:1059C000BFF920460021FFF7D7F801F0B5FA00280B
:1059D00018BF10BD4EF60450CEF200004FF08051BB
:1059E0000160BFF34F8FBFF36F8F10BDB0B590B1A3
:1059F0000D46D1B1044644F62810C2F200000068FA
:105A0000E8B14FF0500080F31188BFF36F8FBFF300
:105A10004F8F00BFFEE74FF0500080F31188BFF3B7
:105A20006F8FBFF34F8F00BFFEE74FF0500080F342
:105A30001188BFF36F8FBFF34F8F00BFFEE700F0F9
:105A40007FF945F2E800C2F2000000682268904247
:105A500002EB050102D2914202D309E0914201D347
:105A6000814205D92160081A0021FFF785F800E07E
:105A7000216001F061FA002818BFB0BD4EF6045055
:105A8000CEF200004FF080510160BFF34F8FBFF3A3
:105A90006F8FB0BD70B50446FFF77AFE40F2D04676
:105AA000002CC2F2000608BF3468251D2846FFF707
:105AB000FBFDA06A18B104F11800FFF7F5FD44F6EC
:105AC0002C10C2F20000016801310160306884428C
:105AD0000CD044F62010C2F20000016801390160C8
:105AE0002046FFF797F9FFF747FC0DE045F2D40099
:105AF000C2F200002946FFF733FE44F62410C2F23A
:105B00000000016801310160FFF766FE45F2B40054
:105B1000C2F200000068E8B13068844218BF70BD6E
:105B200044F62810C2F20000006840B14FF0500067
:105B300080F31188BFF36F8FBFF34F8FFEE74EF6F0
:105B40000450CEF200004FF080510160BFF34F8F40
:105B5000BFF36F8F70BD000045F25001C2F200012B
:105B60000968016045F2E801C2F20001096841607C
:105B70007047000045F2F400C2F20000012101600C
:105B80007047000010B568B10C4640F2D041C2F237
:105B9000000109681831FFF7C5FD20460121FEF715
:105BA000EBFF10BD4FF0500080F31188BFF36F8FF3
:105BB000BFF34F8FFEE70000B0B590B10D4640F245
:105BC000D041C2F20001096814461831FFF7C8FD40
:105BD000002C18BF4FF0FF3528462146FEF7CCFFBA
:105BE000B0BD4FF0500080F31188BFF36F8FBFF34B
:105BF0004F8F00BFFEE7000070B528B3026D04466A
:105C00001AB3E06C884238BF0846012A1CD1E16A09
:105C1000814208BF70BD40F2D042C2F20002126859
:105C2000A2421CD0A269E062002A5CBFC0F1380029
:105C3000A06140F2E846606901EB8101C2F2000612
:105C400006EB8101884214D070BD4FF0500080F304
:105C50001188BFF36F8FBFF34F8F00BFFEE74FF088
:105C6000500080F31188BFF36F8FBFF34F8F00BFD9
:105C7000FEE7251D2846FFF717FD44F63011C2F256
:105C80000001E06A0A68904288BF086000EB80006B
:105C900006EB80002946FFF763FD70BD10B586B0A6
:105CA000002405A804A903AACDE90444FFF70EFDCA
:105CB000DDE9032005990023CDE9010144F6F960EF
:105CC000C0F600001CA1009400F0EEFD45F2440176
:105CD000C2F20001086010B101F0B8F90446601C7E
:105CE00020D0012C1CD14FF0500080F31188BFF35D
:105CF0006F8FBFF34F8F45F24C00C2F200004FF0A0
:105D0000FF31016045F2B400C2F2000001210160E0
:105D100045F2E800C2F200000021016000F066F8E0
:105D200006B010BD4FF0500080F31188BFF36F8FA5
:105D3000BFF34F8FFEE700BF49444C450000000011
:105D400044F62810C2F2000001680131016070477A
:105D500044F62810C2F20000006830B145F2F400A9
:105D6000C2F2000001210160704745F2F400C2F266
:105D70000000002144F6301C0160C2F2000CDCF887
:105D8000001040F2E84201EB8103C2F2000252F837
:105D9000230048B902EB8300A0F11403D9B153F8F2
:105DA000140901390028F9D001EB810002EB8002CF
:105DB00052F8040F4368101D8342136001D15868E4
:105DC0001060106840F2D042C068C2F20002106059
:105DD000CCF8001070474FF0500080F31188BFF3EB
:105DE0006F8FBFF34F8F00BFFEE7000080B582B01A
:105DF0004EF20040CEF200004CF27021C4F20F11BE
:105E0000D0F800294B1C9A4209D14FF0500080F382
:105E10001188BFF36F8FBFF34F8F00BFFEE7D0F83D
:105E200000298A4209D14FF0500080F31188BFF356
:105E30006F8FBFF34F8F00BFFEE7017844F6141257
:105E40000191FF2101700178C2F200028DF8031068
:105E50009DF8031001F05001117044F61811C2F2C0
:105E6000000107220A609DF90320B2F1FF3F0CDC1C
:105E70000A6800BF9DF80330013A5B008DF80330DB
:105E80009DF90330002BF5D40A600A68032A2DD14E
:105E90004FF4E06303EA02220A6001990170D0F82E
:105EA000201941F47001C0F82019D0F8201941F0F0
:105EB0007041C0F82019FFF7EDFC40F2C000C2F2BB
:105EC000000000210160FFF759FC4EF63470CEF25D
:105ED0000000016841F040410160FFF72FF9FFF732
:105EE00037FFFFF7BBFA002002B080BD4FF0500033
:105EF00080F31188BFF36F8FBFF34F8FFEE7000071
:105F000080B54FF0500080F31188BFF36F8FBFF35F
:105F10004F8F00F043FE30B14EF60450CEF2000039
:105F20004FF080510160002080F3118880BD000097
:105F300010B502460120002100F018F80446FEF7D3
:105F4000F1FF204610BD000010B582B00B4684461C
:105F5000012000210022CDF800C000F02BF80446FB
:105F6000FEF7E0FF204602B010BD0000F0B581B0A2
:105F7000B0B105464843503014460E46FFF7CEFAFE
:105F8000074650B1002007F1500287F84600284626
:105F9000314623460097FEF7D5FF384601B0F0BDE5
:105FA0004FF0500080F31188BFF36F8FBFF34F8F16
:105FB000FEE70000B0B582B068B11D46ABB1F1B9E3
:105FC000EAB14FF0500080F31188BFF36F8FBFF339
:105FD0004F8F00BFFEE74FF0500080F31188BFF3F2
:105FE0006F8FBFF34F8F00BFFEE74FF0500080F37D
:105FF0001188BFF36F8FBFF34F8F00BFFEE751B122
:106000004AB94FF0500080F31188BFF36F8FBFF390
:106010004F8F00BFFEE750230193019B502B0AD105
:10602000069B019C012485F846400095FEF78AFFF7
:10603000284602B0B0BD4FF0500080F31188BFF386
:106040006F8FBFF34F8F00BFFEE7000070B5F8B150
:1060500004460E46FFF79CFB2068D4E90F1200258A
:1060600002FB0103013901FB0201A563C4E901033D
:10607000FF20E16084F8440084F8450004F110003A
:106080007EB1FFF73FFB04F12400FFF73BFB18E074
:106090004FF0500080F31188BFF36F8FBFF34F8F25
:1060A000FEE7016869B100F0FFFE50B14EF6045002
:1060B000CEF200004FF080510160BFF34F8FBFF36D
:1060C0006F8FFFF789FB012070BD00002DE9F04FB5
:1060D00083B00292B8B11D460E460446E9B1022DC6
:1060E00003D1E06B012840F09A8000F033FD00BB43
:1060F0000298F0B14FF0500080F31188BFF36F8F1A
:10610000BFF34F8FFEE74FF0500080F31188BFF3CD
:106110006F8FBFF34F8F00BFFEE7206C0028DED0EB
:106120004FF0500080F31188BFF36F8FBFF34F8F94
:10613000FEE7FFF72DFBA06B022D58D0E16B8842E4
:1061400055D304F1100801206F464FF0000B0DF1FC
:1061500008094FF0805A00BF0299002900F07B80A7
:10616000C00702D03846FFF7F7FCFFF735FBFFF713
:10617000E7FDFFF70DFB94F84400FF2808BF84F803
:1061800044B094F84500FF2808BF84F845B0FFF7F5
:1061900023FB3846494600F00FFB00285ED120461D
:1061A000FEF7BEFFA0B102994046FFF7EBFC204688
:1061B000FFF77AF900F0C0FE78B94EF60450CEF23F
:1061C0000000C0F800A0BFF34F8FBFF36F8F04E053
:1061D0002046FFF769F900F0AFFEFFF7D9FAA06B90
:1061E000022D04D0E16B88424FF00000B4D220466B
:1061F00031462A46FEF7D0FD54F8241FC9B1204687
:1062000000F052FE08B34EF60450CEF200004FF0FC
:1062100080510160BFF34F8FBFF36F8F15E04FF0D8
:10622000500080F31188BFF36F8FBFF34F8F00BF13
:10623000FEE750B14EF60450CEF200004FF0805110
:106240000160BFF34F8FBFF36F8FFFF7C5FA0120D7
:1062500003B0BDE8F08FFFF7BFFA04E02046FFF778
:1062600023F900F069FE002003B0BDE8F08F0000C4
:106270002DE9F04381B0E8B11E46914605460F4630
:1062800009B3022E02D1E86B012837D1FFF71CFBBE
:10629000EFF311884FF0500080F31188BFF36F8F38
:1062A000BFF34F8FA86B022E19D0E96B884216D32B
:1062B00000203FE04FF0500080F31188BFF36F8F54
:1062C000BFF34F8FFEE7286C0028DAD04FF0500064
:1062D00080F31188BFF36F8FBFF34F8FFEE795F800
:1062E0004540A86B284639463246FEF755FDFF2C3F
:1062F0000DD0601C85F8450001201BE04FF05000D8
:1063000080F31188BFF36F8FBFF34F8FFEE755F80F
:10631000240F70B1284600F0C7FD0146B9F1000F07
:106320004FF0010006D000291CBF0120C9F8000071
:1063300000E0012088F3118801B0BDE8F08300007F
:10634000B0B5A8B18568044600F0FEFB85421CBFCD
:106350000020B0BDE0680138E0601CBF0120B0BD86
:106360002046002100220023FFF7B0FE0120B0BD2F
:106370004FF0500080F31188BFF36F8FBFF34F8F42
:10638000FEE700002DE9F04F85B0049298B10C466D
:106390000546002900F0A58000F0DCFBA8B90498B0
:1063A00098B14FF0500080F31188BFF36F8FBFF3A7
:1063B0004F8F00BFFEE74FF0500080F31188BFF30E
:1063C0006F8FBFF34F8F00BFFEE705F1240005F18B
:1063D0001009019002AF0DF1100A4FF000080AE019
:1063E0002846FFF761F800F0A7FD2846FEF78CFE6F
:1063F000002840F08480FFF7CBF9D5F838B0BBF126
:10640000000F1DD028462146FEF7B2FCABF101007B
:10641000A863286970B1484600F046FD50B14EF6B9
:106420000450CEF200004FF080510160BFF34F8F57
:10643000BFF36F8FFFF7D0F900200126A0B95FE00E
:10644000049850B1B8F1000F02D13846FFF784FB31
:106450004FF00108012038B952E0FFF7BDF90026DE
:10646000002000284CD000BFFFF7B6F9FFF768FC0A
:10647000FFF78EF995F84400FF2804BF002085F847
:10648000440095F84500FF2804BF002085F845002A
:10649000FFF7A2F93846514600F08EF900289FD147
:1064A0002846FEF731FEB0B104990198FFF76AFB68
:1064B0002846FEF7F9FF00F03FFD00289BD14EF67D
:1064C0000450CEF200004FF080510160BFF34F8FB7
:1064D000BFF36F8F8FE72846FEF7E6FF00F02CFD35
:1064E00089E7286C00283FF457AF4FF0500080F345
:1064F0001188BFF36F8FBFF34F8F00BFFEE70026F9
:10650000304605B0BDE8F08F2DE9F04381B000B30F
:10651000914605460E4631B3FFF7D6F9EFF31188E1
:106520004FF0500080F31188BFF36F8FBFF34F8F90
:10653000AC6B24B395F8447028463146FEF718FC3E
:10654000601EFF2FA8631CD0781C85F84400012032
:106550002AE04FF0500080F31188BFF36F8FBFF334
:106560004F8F00BFFEE7286C0028D5D04FF05000B9
:1065700080F31188BFF36F8FBFF34F8FFEE70020CA
:1065800012E055F8100F70B1284600F08DFC01465E
:10659000B9F1000F4FF0010006D000291CBF012007
:1065A000C9F8000000E0012088F3118801B0BDE8BF
:1065B000F08300002DE9F04F85B0049158B10446F6
:1065C000006C90B14FF0500080F31188BFF36F8FD3
:1065D000BFF34F8FFEE74FF0500080F31188BFF3F9
:1065E0006F8FBFF34F8F00BFFEE700F0B3FA50B9D3
:1065F000049840B14FF0500080F31188BFF36F8FC3
:10660000BFF34F8FFEE704F1240004F11005019061
:106610004FF0000802AF0DF1100A4FF000094FF0E3
:10662000000B0AE02046FEF73FFF00F085FC204605
:10663000FEF76AFD002840F07F80FFF7A9F8A06B05
:10664000F0B10138A063206810B9FFF70DF8A06021
:10665000286870B1284600F027FC50B14EF604506F
:10666000CEF200004FF080510160BFF34F8FBFF3B7
:106670006F8FFFF7B1F801260020B8B96FE000BFB7
:10668000049850B1BBF1000F02D13846FFF764FA0D
:106690004FF0010B012048B961E0B9F1000F62D160
:1066A000FFF79AF800200026002858D0FFF794F84A
:1066B000FFF746FBFFF76CF894F84400FF2808BF8B
:1066C00084F8448094F84500FF2808BF84F845808A
:1066D000FFF782F83846514600F06EF80028A1D145
:1066E0002046FEF711FD28B92046FEF7DDFE00F03A
:1066F00023FCA2E7206838B9FFF74AF8A06800F049
:1067000089FB8146FFF768F804990198FFF73AFA88
:106710002046FEF7C9FE00F00FFC00287FF48DAF85
:106720004EF60450CEF200004FF080510160BFF3EE
:106730004F8FBFF36F8F80E7B9F1000F0ED0FFF7D7
:1067400027F82046FEF782FBA1680246084611465C
:10675000FFF752FAFFF740F8002600E00026304627
:1067600005B0BDE8F08F4FF0500080F31188BFF303
:106770006F8FBFF34F8F00BFFEE7000070B568B1A9
:10678000866804460D4600F0DFF986420FD02046A9
:106790002946FFF70FFF58B9002070BD4FF0500099
:1067A00080F31188BFF36F8FBFF34F8FFEE7012097
:1067B000E1680131E16070BDB0B5D0B10D4611B3F3
:1067C0000446FEF7E5FF45F2E800C2F2000001686A
:1067D0002868421C21D045F250036268C2F20003CF
:1067E000D3F800C091421AD323689C4517D00124E6
:1067F00022E04FF0500080F31188BFF36F8FBFF39A
:106800004F8F00BFFEE74FF0500080F31188BFF3B9
:106810006F8FBFF34F8F00BFFEE700240CE0891A93
:10682000884206D9401A28602046FFF795F90024CF
:1068300002E0002001242860FEF7CEFF2046B0BD14
:106840002DE9F04383B007469000984615468946E7
:10685000FEF764FE78B106465C20FEF75FFE38B1B5
:106860000446066354B94FF0FF3003B0BDE8F0832F
:106870003046FEF7C9FF0024002CF4D0DDE90A10F1
:10688000002284F85920CDE90010384649462A46AE
:1068900043460294FEF766FB2046FEF7ADF9012061
:1068A00003B0BDE8F083000070B586B00B9CCCB19E
:1068B0000C9E06B35C250495049D5C2D25D1049D9A
:1068C000DDF828C0022586F8595005AD3463CDE9BE
:1068D00000C50296FEF746FB3046FEF78DF9059897
:1068E00006B070BD4FF0500080F31188BFF36F8F7A
:1068F000BFF34F8FFEE74FF0500080F31188BFF3D6
:106900006F8FBFF34F8F00BFFEE74FF0500080F353
:106910001188BFF36F8FBFF34F8F00BFFEE70000FA
:10692000F0B581B0D0B11D46174604460E46FEF7BD
:106930002FFF002D1CBF606D286094F858000221C5
:10694000042F84F8581012D80125DFE807F023033C
:106950001C262000616D314361651FE04FF050003F
:1069600080F31188BFF36F8FBFF34F8FFEE7616D28
:10697000013113D04FF0500080F31188BFF36F8FB7
:10698000BFF34F8FFEE7616D0131616506E00228BC
:1069900003D1002501283CD103E0666501250128CB
:1069A00037D1261D3046FEF77FFE44F63011C2F285
:1069B0000001E06A0A68904288BF086040F2E8413E
:1069C00000EB8000C2F2000101EB80003146FEF7CF
:1069D000C7FEA06A48B14FF0500080F31188BFF3A2
:1069E0006F8FBFF34F8F00BFFEE740F2D041C2F27E
:1069F0000001E06A0968C96A88420AD94EF6045063
:106A0000CEF200004FF080510160BFF34F8FBFF313
:106A10006F8FFEF7E1FE284601B0F0BD2DE9F04191
:106A200020B31D46174604460E46FEF74DFFEFF312
:106A300011884FF0500080F31188BFF36F8FBFF3C0
:106A40004F8F002D1CBF606D286094F85800022104
:106A5000042F84F8581012D80125DFE807F023032B
:106A60001C262000616D314361651FE04FF050002E
:106A700080F31188BFF36F8FBFF34F8FFEE7616D17
:106A8000013113D04FF0500080F31188BFF36F8FA6
:106A9000BFF34F8FFEE7616D0131616506E00228AB
:106AA00003D10025012849D103E0666501250128AD
:106AB00044D1A06A48B14FF0500080F31188BFF371
:106AC0006F8FBFF34F8F00BFFEE744F62810C2F26E
:106AD0000000006830B145F2600004F11801C2F214
:106AE000000015E0261D3046FEF7DEFD44F63011AD
:106AF000C2F20001E06A0A68904288BF086040F272
:106B0000E84100EB8000C2F2000101EB8000314659
:106B1000FEF726FE40F2D041C2F20001E06A0968A9
:106B2000C96A88420AD9069800281CBF0121016061
:106B300045F2F400C2F200000121016088F31188DF
:106B40002846BDE8F081000040F2D040C2F20000CB
:106B50000068704745F2B400C2F2000000680028E7
:106B600004BF0120704744F62810C2F200000068FC
:106B7000B0FA80F0400940007047000045F2E8009C
:106B8000C2F200000068704780B5FEF79DFE45F236
:106B9000E800C2F20000006880BD00002DE9F04F5F
:106BA00081B044F62810C2F20000006840B145F2FE
:106BB0005C00C2F20000016800240131016092E033
:106BC00045F2E800C2F2000001684E1C066021D3C5
:106BD00040F2D840C2F200000168096849B14FF0A4
:106BE000500080F31188BFF36F8FBFF34F8F00BF4A
:106BF000FEE740F2E042C2F200020168136803605F
:106C000045F250001160C2F20000016801310160DC
:106C1000FEF7B2FB45F24C01C2F20001086840F2F7
:106C2000D04A40F2E8488642C2F2000AC2F20008A6
:106C300001D2002445E040F2D847C2F2000738688C
:106C40000024006898B344F6301BC2F2000B19E030
:106C5000D9F82C00DBF80010884288BFCBF8000080
:106C600000EB800008EB80002946FEF779FDD9F89B
:106C70002C00DAF80010C96A3A68884228BF01245B
:106C80001068B8B13868C068D0F80C904D4655F817
:106C9000040F864210D32846FEF706FDD9F82800D7
:106CA0000028D5D009F11800FEF7FEFCD0E74FF020
:106CB000FF3005E04FF0FF3045F24C01C2F2000119
:106CC0000860DAF80000C06A00EB800058F8200085
:106CD000012845F2F400C2F2000088BF01240068D8
:106CE000002818BF0124204601B0BDE8F08F000045
:106CF0002DE9F0411E46154688460746FEF748FD39
:106D000040F2D044C2F20004206890F858000228F3
:106D100019D02068416D21EA0701416520684FF0D4
:106D2000010180F8581076B130460121FDF724FFAB
:106D30004EF60450CEF200004FF080510160BFF3D8
:106D40004F8FBFF36F8FFEF747FDFEF721FD15B1A3
:106D50002068406D28602068002590F858100020B9
:106D6000022905D1216801254A6D22EA08024A65F7
:106D7000216881F85800FEF72FFD2846BDE8F08114
:106D8000B0B580B1044640F2D040C2F200000068C5
:106D9000A0420AD04FF0500080F31188BFF36F8FEC
:106DA000BFF34F8FFEE70020B0BD206D38B3013830
:106DB00020654FF0000018BFB0BDE16AE26C91425F
:106DC0001CD0251D2846FEF76FFCE06CC0F1380191
:106DD000A16144F63011E062C2F200010A689042FB
:106DE00088BF086040F2E84100EB8000C2F2000179
:106DF00001EB80002946FEF7B3FC0120B0BD4FF047
:106E0000500080F31188BFF36F8FBFF34F8F00BF27
:106E1000FEE70000F0B581B000B340F2D046C2F208
:106E200000060446C06A3168C96A884219D2A1695D
:106E3000002904D43168C96AC1F13801A16140F266
:106E4000E847616900EB8000C2F2000707EB8000B1
:106E500081420FD03068C06AE06221E0002001B0BA
:106E6000F0BDE16C3068C26A0020914238BF012059
:106E700001B0F0BD251D2846FEF716FC306844F62B
:106E80003011C06AC2F20001E0620A68904288BF15
:106E9000086000EB800007EB80002946FEF760FCED
:106EA000012001B0F0BD0000B0B5C068C5687DB17B
:106EB00005F118042046FEF7F7FB44F62810C2F24D
:106EC0000000006868B145F26000C2F200001DE0F9
:106ED0004FF0500080F31188BFF36F8FBFF34F8FD7
:106EE000FEE72C1D2046FEF7DFFB44F63011C2F210
:106EF0000001E86A0A68904288BF086040F2E841F1
:106F000000EB8000C2F2000101EB80002146FEF799
:106F100027FC40F2D041C2F20001E86A0968C96A60
:106F2000884291BF002045F2F401C2F20001012025
:106F300088BF0860B0BD00002DE9F04F81B044F675
:106F40002814C2F20004206868B1FEF721FC206812
:106F500001382060206880B10024FEF73DFC204607
:106F600001B0BDE8F08F4FF0500080F31188BFF3FF
:106F70006F8FBFF34F8F00BFFEE744F62010C2F2C1
:106F80000000006800285DD045F26006C2F20006ED
:106F9000306845F2F408C2F2000890B344F63017A6
:106FA00040F2E84940F2D04BC2F20007C2F20009B9
:106FB000C2F2000B4FF0010AF068C56805F1180035
:106FC000FEF772FB2C1D2046FEF76EFBE86A39685F
:106FD000884288BF386000EB800009EB80002146C2
:106FE000FEF7BEFBE86ADBF80010C96A884228BFDA
:106FF000C8F800A030680028DED1002D18BFFEF7C9
:10700000BBF945F25C04C2F20004256855B10126C3
:10701000FFF7C4FD002818BFC8F80060013DF7D194
:1070200000202060D8F8000070B14EF60450CEF277
:1070300000004FF080510160BFF34F8F0124BFF378
:107040006F8F8AE7002488E7002486E780B586B042
:10705000FDF728FE45F2EC00C2F20000006808B31C
:107060000020CDE9040005A804A903AAFEF73CFB13
:10707000DDE903200221DDF814C0CDE9001045F25E
:107080009140C0F600000CA10023CDF808C0FFF726
:107090000BFC45F2F001C2F20001086010B10120C2
:1070A00006B080BD4FF0500080F31188BFF36F8FA2
:1070B000BFF34F8FFEE700BF546D7220537663001D
:1070C00010B584B0A8B145F2EC04C2F200048446C5
:1070D0002068C0B10529CDE90012CDF808C015DC43
:1070E000FFF738FD01462068022916D1069A694645
:1070F00015E04FF0500080F31188BFF36F8FBFF39E
:107100004F8F00BFFEE7002004B010BD69461A464D
:107110000023FFF7ADF804B010BD6946002200233C
:10712000FEF7D4FF04B010BD4100080218BF0420D0
:107130000A0E18BF40F001004FF07F4232EA010111
:1071400008BF40F00200012808BF0520704700007A
:1071500010B52DED040B86B09DED060B10EE100A58
:1071600010EE901A8DED000B002818BF0120084387
:1071700020F00040C0F17F6000F1E040C00F21D15D
:107180009DED080B10EE101A10EE900A8DED000B1D
:10719000002918BF0121084320F00040C0F17F60A2
:1071A00000F1E040C00F0DD129490798B1EB400F25
:1071B00004BF0698002842D00998400004BF0898F0
:1071C00000283CD09DED080B53EC102B9DED060BD9
:1071D00051EC100B00F08CFCCDE902019DED020B8F
:1071E00040F2FF7110EE900A8DED000B31EA105065
:1071F00021D00798039900F0004001F00041884237
:1072000019D09DED080B8DED040B9DED020B8DED5E
:10721000000B10EE900A059961F31E0005909DED9C
:10722000041B9DED020B51EC110B53EC102B00F0E5
:107230000DFDCDE902019DED020B0AB010BD01204C
:10724000F9F738F90AB0BDE8104000F0C1B8000005
:107250000000E0FF00B510EE101A2DED028B81B09A
:107260004D4A6846B2EB410F3CD94FF0E640B0EBD7
:10727000410F94BF00204FF0FF3000900098B0EE17
:10728000408A00285FDB28EE080ADFED440A9FED04
:10729000441A00EE201ADFED430A40EE010A9FED8A
:1072A000421A00EE201ADFED410A10F0010F40EE05
:1072B000010A9FED3F1A00EE201A61EE000AB0EEBF
:1072C000480A08EE200A02BF01B0BDEC028B00BDE7
:1072D000BFEE001A01B0C1EE000ABDEC028BB0EEA9
:1072E000600A00BD334B21F00042934228D911F0CF
:1072F000004FDFED310A20EE201ADFED300A19BF12
:1073000031EE601A71EE200A31EE201A71EE600A39
:10731000BDEEE01A11EE100A9FED291A00F00300ED
:1073200000EEC10A9FED271A009000EEC10A9FED02
:10733000261A00EEC10A9FED251A00EEC10A9DE74C
:1073400000F06AF89AE718EE100A4000B0F17F4F9B
:107350000DD218EE100AFFF7E7FE042808BF00F070
:1073600053F8B0EE480A01B0BDEC028B00BD09D164
:107370000120F9F79FF801B0BDEC028B5DF804EB3A
:1073800000F03AB801B0B0EE480ABDEC028B5DF8EF
:1073900004EB00F02DB80000B61F927EBCE9223C41
:1073A0000B6D063B8A76CE3CACB5593D35A1083E07
:1073B00029AAAA3E490E494683F9223F0000004B04
:1073C0000000C93F00A0FD390020A2331A61342C0F
:1073D0009FED050B10B553EC102B51EC100B00F08A
:1073E0009FF941EC100B10BD0000000000000000F0
:1073F00030EE000A70470000DFED020A80EEA00ABE
:1074000070470000000000009FED020A20EE000A15
:1074100070470000000000102DE9F0014FF07F429E
:10742000B2EB410F9FBF4FF0FF310160BDE8F001AB
:1074300070474FF0004242EA0123C1F3C752783A45
:10744000551112F01F0C434CCCF120067C44C1F3C3
:10745000C752A2F178024FEA621204EB820254F89A
:10746000254008BFD2E9015612D0556804FA0CF441
:1074700025FA06F73C43976805FA0CF527FA06F853
:10748000D26807FA0CFCF24045EA08054CEA02060D
:10749000A4FB034CA5FB0352A6FB03631D449D42C2
:1074A00034BF012600261319334416B1934202D982
:1074B00003E0934201D2012200E00022624402F183
:1074C000200C9206DC0C42EA443200EE102A5B03E8
:1074D000DFED210AF8EEC01A00EE103A4FEA9C1CCC
:1074E00011F0004FB8EE400AC0F800C020EE201A9C
:1074F00000EE105ADFED190AB8EE400A20EE200A1D
:1075000071EE810A70EE800A10EE902A02F5006298
:107510006FF30B0200EE902A70EEE11A31EEC11A01
:10752000DFED101A30EE411A9FED0D0A20EE800AB1
:1075300001EE210A9FED0C1A00EE810A04BFBDE89E
:10754000F0017047CCF180510160BDE8F001B1EE6F
:10755000400A7047580B0000000000360000802CE5
:1075600022AAFD29DB0FC92F0000C92F21F00042FC
:1075700001F00043A2F16052B2F5801F28BFD2F1A2
:107580007F6C0BD95FEA001C43EAC20242EB5070E9
:1075900018BF704728BF20F001007047B2F5801F68
:1075A000BCBF184670474FEA410C1CF5001F02D2C1
:1075B000084600F0F3BC70B500F04CFA00000089FA
:1075C000FFF7F6BF4FF00040A0F5800070470000C5
:1075D00010B591EA030F48BF83F0004300F14A83DE
:1075E000841A71EB030C05D2121943EB0C03001B38
:1075F00061EB0C014FEA1154A4EB135CDFF81CE1C2
:107600001EEA430F18BF9EEA445F00F0748021EA2F
:10761000045123EA0E0343F48013DCF1200E32D32D
:1076200022FA0CFE10EB0E0023FA0CFE41EB0E01C9
:10763000CCF1200E03FA0EFE10EB0E00CCF1200E62
:1076400051F10001B1F5801F32D201EB045112FA61
:107650000EF2BDE8104058BF7047401C38BF5FEACB
:10766000420218BF7047002814BF20F0010041F10A
:1076700000014FEA410313F5001F38BF7047A1F125
:10768000C04100F0DDBA012A43EB0302ACF1200C4B
:10769000DCF11F0E32BF4FF0000E23FA0CF310EB9B
:1076A000030041EB0451B4EB115FD0D0A1EB0451C6
:1076B00001F58011490801EB04515FEA30000ED357
:1076C00050F1000038BF12FA0EFE08D1BDE810409C
:1076D000C9E7401C38BF5FEA4202CAD1C3E7BDE830
:1076E00010404FEA410313F5001F38BF7047A1F166
:1076F000C04100F0A5BA9EEA445F08D011EA5E0FCF
:10770000BDE8104004BF01F0004100207047BDE813
:10771000104070B500F09EF964FBBE3E0000E0FF33
:107720002DE9C04130B4DFF8A4C23CEA111418BFFF
:107730003CEA131400F0ED801CEA111481EA030501
:1077400044EAD57418BF1CEA131500F0C880A4EBF6
:10775000050404F17F7404F500344FF0004545EA58
:10776000C12145EAC32341EA505143EA52534FEA4B
:10777000C0204FEAC222994208BF904200F09D808B
:107780004FEA13650FF24416765D4FEA134506FB88
:1077900005F7C7F1807706FB07F74FEAD737A7FB56
:1077A00003687642A7FB06CEC8F5803838BFA8F13B
:1077B000010807FB08E6A6FB028C4FF0000EE6FB73
:1077C00003CEDCF1000CCEF1004E38BFAEF1010E5D
:1077D000A6FB0C584FF00007E6FB0E87A1FB08C67E
:1077E000A0FB07CE16EB0E064FF0000545F1000595
:1077F000E1FB076515F1E04E7EBFA4F580345FEA3A
:1078000046066D4116F1800745F100054FEA17273E
:1078100047EA05674FEA15254FEA0666A6F1DE46F8
:10782000B6F1805F20D9384605EBC47124F0010C15
:1078300001EB0C11BCF1FE6F02D8F0BCBDE8008179
:1078400024425CBF01F5801E9EEAC47F02D4F0BCD6
:10785000BDE80081244200F13980A1F1C041F0BCB3
:10786000BDE8004100F0ECB94FEAD02040EA4150B9
:107870004FEAD1214FEAD22242EA43524FEAD323C0
:10788000A7FB028607FB036605FB02661EEA0E0FD6
:1078900058BFA6EB0056B6EB00564FEA520E4EEA22
:1078A000C37E18EB0E0E56EB530EBCD518EB020838
:1078B0005E417F1C55F10005B5E74FF480154FF090
:1078C00000074FF000064FF00008ACE701F1C0419F
:1078D00001F000414FF00000F0BCBDE800810CEA6F
:1078E000131511EA0C1F00D00CE013EA0C1F00F076
:1078F00026804FF0000081EA030101F00041F0BC56
:10790000BDE80081F0BCBDE8004181EA030100F060
:1079100097B9F0BCBDE8004170B500F09BF800BF1E
:10792000097EFC3E00F007B84FF0000081EA030139
:1079300001F00041704781EA030100F081B9F0BC19
:10794000BDE8004122494FF000007047FFFDFBF900
:10795000F7F5F4F2F0EEEDEBE9E8E6E4E3E1E0DE82
:10796000DDDBDAD8D7D5D4D3D1D0CFCDCCCBCAC8F4
:10797000C7C6C5C4C2C1C0BFBEBDBCBBBAB9B8B71B
:10798000B6B5B4B3B2B1B0AFAEADACABAAA9A8A80E
:10799000A7A6A5A4A3A3A2A1A09F9F9E9D9C9C9BDC
:1079A0009A99999897979695959493939291919087
:1079B0008F8F8E8E8D8C8C8B8B8A89898888878718
:1079C0008685858484838382828181800000FF078D
:1079D0000000F87F4FEA1153A3F58063D3F11E0333
:1079E000A8BFD3F1200C08DB4FF0004242EAC122CD
:1079F00052EA505232FA03F0704709420BD4102B6E
:107A0000C4BF0020704703F5787CBCF1FF3F05D070
:107A10004FF0FF3070474FF00000704770B500F036
:107A200019F800BF4992248000207047F0E7B0FAAF
:107A300080F310FA03F10AD0C3F11D0303F580634C
:107A40004FEA03524FEA415002EBD12170474FF009
:107A5000000070470EF1020E2EF0030E5EF8046B6C
:107A6000364205D4012A43EB030515F5001F12D851
:107A7000012841EB010C1CF5001F0CD80ED14FEA78
:107A8000D17C0CEB4C0C0CF1020C15F5001F08BF5F
:107A90004CEBD37C04E04FF0080C01E04FEAD37CC0
:107AA0000CEB4C0526FA05F606F00706B6F1040CB9
:107AB00006D20EEB860CBDE870404CF0010C60471E
:107AC000DFE80CF0090B02024FF00041A1F50021A4
:107AD0004FF0000070BD19461046012851EB01041B
:107AE00018BFD4F5001484BF002001F0004170BD20
:107AF00070B5DFF844C13CEA111418BF3CEA131515
:107B000000F08F8011F1004F0CEA11141CEA1315DC
:107B100068BF45F0050518BF11EA0C1F00F0798019
:107B200021EA4C1123EA4C1341F4801143F48013F1
:107B30002E46A5F58035AC423DDDA4F58036801A91
:107B4000994109D54042C1F1000134BFB1F10101B1
:107B5000B1F1000185F0010511F4F01F08D011F416
:107B6000801FE8D1400041EB0101A4F58034F6E725
:107B700021F00041B1FA81F6202E04BFB0FA80FE58
:107B80000EF12006A6F10B06A4EB0644B6F1200E7A
:107B90000CD2C6F1200E01FA06F120FA0EF641EAE7
:107BA0000601CEF1200600FA06F003E000FA0EF11D
:107BB0004FF00000BFE750EA410E23D04FEA244EB9
:107BC000BEEB254F0FDB994208BF904204D00AD389
:107BD000520043EB0303B0E74FEA1646B6EB144FEF
:107BE00008BF85F00105B4F5803401EB041181EA8A
:107BF000C57100DB70BD01F1C04101F000414FF0E3
:107C0000000070BD4FEA45714FF0000001F00041E7
:107C100070BD1CEA131F09D04FF0000001F00041B5
:107C200070BDFFF717FF00BFEDFFFF3EBDE87040DE
:107C300002494FF0000070470000FF070000F87F86
:107C40000808A0F500114FEA3101704710B591EA1C
:107C5000030F81F000413FF5C3AC83F0004300F017
:107C600009B8000010B591EA030F48BF83F0004344
:107C70003FF5B6AC841A71EB030C07D28CF0004CC4
:107C8000121943EB0C03001B61EB0C014FEA11547A
:107C9000A4EB135CDFF8A4E11EEA430F18BF9EEAD1
:107CA000445F00F0B48021EA045123EA6E0352429B
:107CB000C3EB6E0338BF5B1EDCF1200E25D322FA26
:107CC0000CFE10EB0E0043FA0CFE41EB0E01CCF162
:107CD000200E03FA0EFE10EB0E00CCF1200E51F137
:107CE000000129D401EB045112FA0EF2BDE8104054
:107CF00058BF7047401C1CBFB2F1004F70470028AE
:107D00000CBF491C20F00100704712EB020E43EB40
:107D1000030218BF4FF0010E4EEA4202ACF1200CF4
:107D2000DCF11E0E56D943FA0CFE10EB0E00CCF11E
:107D30001E0E51F1FF31D5D50EF1010E12FA0EFED5
:107D4000404141EB010101EB445C5FEA5C5C10D90E
:107D500001EB045110EBDE7038BFBEF1004FBDE8FF
:107D6000104018BF704700280CBF491C20F00100CC
:107D7000704734D24FEAD42C24F4006411F500117A
:107D80001BD0B1FA81F20B3AA41AA41ED2F120033F
:107D9000914030FA03F31943904001EBCC7101EBB1
:107DA0000451002CBDE81040A8BF704701F1C0414C
:107DB00001F000414FF000007047B0FA80F310FA74
:107DC00003F102D1BDE810407047E41A173C4805A2
:107DD000C90AE2E701EB0451BDE8104070474910C1
:107DE0004FEA300001EB0451BDE8104002E04FF0D3
:107DF000000170474A0008BF0042F8D0B2F5001FEA
:107E000028BF704701F000414FF0000070479EEA24
:107E1000445F07D011EA5E0FBDE8104004BF0021A7
:107E200000207047BDE8104070B5FFF713FE00BF9B
:107E300040DFF63E104683F0004170470000E0FF4F
:107E400043004FEAD30C4FEA3C0C43401FBF4007AE
:107E50000CF1605113F0FE4F70471CF0006F03D11E
:107E60000CF00041002070470CF0004343EA5070D2
:107E700040EACC0010B500F03EF800BF00000092D0
:107E80004FEA0001FFF7DCBE4FF00041A1F50021F1
:107E90004FF0000070474FF07E5209E011F00042B1
:107EA00004D54042C1F1000138BF491E42F07E5264
:107EB00002F170620B0012BF20235FEA00017047DD
:107EC000B1FA81FC01FA0CF1A3EB0C0320FA03FCDC
:107ED00041EA0C0102EBC352C3F1200310FA03FC88
:107EE0005CEA416C42EB112018BF5FF0806C28BF48
:107EF00020F0010070470EF1020E2EF0030E5EF826
:107F0000044B244204D44FEA4102B2F17F4F11D80E
:107F10004FEA4003B3F17F4F0CD80ED14FEAD07C2B
:107F20000CEB4C0C0CF1020CB2F17F4F08BF4CEB88
:107F3000D17C04E04FF0080C01E04FEAD17C0CEB5F
:107F40004C0324FA03F404F00704B4F1040C06D241
:107F50000EEB840CBDE810404CF0010C6047DFE8EC
:107F60000CF0070802024FF00040A0F5800010BDA1
:107F70000846420018BFD2F1807288BF00F000406E
:107F800010BDF1EE100A4FF6FF71C0F2C03120EAC9
:107F9000010040F04070E1EE100A7047FF2141EA15
:107FA000D050C00570470000000000006E83F9A2A9
:107FB0002915444ED15727FCC0DD34F5999562DB75
:107FC0004190433CAB6351FE000000000000000004
:107FD000010203040607080900000000010203046F
:107FE0008A8000080000000000000000000000007F
:107FF000000000000004000030000000000000004D
:10800000000000007C80000800000000000000006C
:108010000000000000000000000400001800000044
:1080200000000000000000007F8000080000000049
:108030000000000000000000000000000008000038
:108040001800000000000000000000007080000820
:108050000000000000000000000000000000000020
:1080600000020000180000000000000000000000F6
:1080700064656661756C745461736B007263007340
:10808000686F6F745F6374726C005461736B5F49E7
:108090006E697400B880000800000020C80000006D
:1080A000C401000880810008C8000020305600008C
:1080B000E0010008000000000024F400DB0F493F4D
:1080C000CDCC4C3E04000100010201000000010083
:1080D0000202010100000100030200000100000093
:1080E0000000803FCDCC4C3FCDCC4C3DCDCCCC3DE9
:1080F000CDCCCC3D6666663F0000F041000080BFFD
:108100000000803F00008040CDCCCC3E0AD7233D0C
:108110000000803E0000803E00002042000080BF42
:108120000000803F0000803FCDCCCC3DCDCC4C3D0D
:10813000CDCC4C3F0000003F000080BFDB0FC940AA
:108140000000803F0000C03F9A99993E0000003F28
:10815000CDCC4C3E6666663F000080BF000080BF0D
:108160000000F0410000F0410000F0410000F0414B
:108170000100000010000000AAAAAAAA0000000046
:040000050800018965
:00000001FF
